:020000040800F2
:10000000B80C0020ED010008355300083544000805
:10001000A5520008F5090008E15F00080000000093
:10002000000000000000000000000000B9530008BC
:10003000290A000800000000B55300080555000813
:10004000070200080702000807020008070200086C
:10005000070200080702000807020008070200085C
:10006000070200080702000807020008F909000853
:10007000050A0008110A00081D0A00080702000806
:10008000070200080702000807020008070200082C
:10009000070200080702000807020008070200081C
:1000A000070200080702000807020008070200080C
:1000B0001D55000845550008070200080702000802
:1000C00007020008070200080702000807020008EC
:1000D00007020008070200080702000807020008DC
:1000E0002D0A00080702000807020008070200089E
:1000F00007020008070200080702000807020008BC
:1001000007020008070200080702000807020008AB
:10011000070200080702000807020008070200089B
:10012000070200080702000807020008070200088B
:10013000070200080702000807020008070200087B
:10014000070200080702000807020008070200086B
:10015000070200080702000807020008070200085B
:10016000070200080702000807020008070200084B
:10017000070200080702000807020008070200083B
:10018000070200080702000807020008070200082B
:10019000070200080000000007020008070200082C
:1001A000070200080702000807020008070200080B
:1001B00007020008070200080702000807020008FB
:1001C00007020008070200080702000807020008EB
:1001D0000702000807020008DFF80CD000F01AFB45
:1001E0000048004735600008B80C002006488047EA
:1001F00006480047FEE7FEE7FEE7FEE7FEE7FEE70C
:10020000FEE7FEE7FEE7FEE709550008D901000812
:100210002DE9F05F0546002092469B46884606463B
:10022000814640241BE0284641464746224600F0CE
:10023000F8F953465A46C01A914110D31146184650
:10024000224600F0DFF92D1A67EB01084F462246DF
:100250000120002100F0D6F917EB00094E41201EC5
:10026000A4F10104DFDC484631462A464346BDE896
:10027000F09FD2B201E000F8012B491EFBD270477B
:100280000022F6E710B513460A4604461946FFF762
:10029000F0FF204610BD2DE9FE4F804681EA0300A5
:1002A000C00F0C46009021F0004123F00045B8EB50
:1002B0000200A94105D24046214690461C460B4605
:1002C000024623F00040104347D0270DC7F30A0031
:1002D000C3F30A510290401A019040286BDAC3F32D
:1002E000130040F4801B0098924620B10023D2EB0B
:1002F000030A63EB0B0B01985946C0F140025046CC
:1003000000F080F906460D4650465946019A00F025
:1003100098F910EB08006141002487EA115284EA41
:10032000E7731A4340D0009A62B3019A012A4FEA58
:10033000075215DC001B61EB02014FF0004202EA9C
:100340000752CDE90042001C41F5801132462B4690
:1003500000F0CFF903B0BDE8F08F40462146F9E741
:10036000001B61EB0201001C41F5801300185B418A
:100370002018A2F5001747EB030140EAD570B61923
:100380006D4111E06D084FEA360645EAC0754FEA47
:100390000752001B61EB0201001C41F58011490866
:1003A0004FEA30000019514132462B4603B0BDE8F8
:1003B000F04F00F08FB90098012240000023D0EBED
:1003C000020263EBE073009821464FEAE074B8EB59
:1003D000000061EB0401E9E783F000435BE781F093
:1003E000004158E72DE9FE4F81EA030404F0004480
:1003F00021F0004100944FF0000B23F0004350EA3D
:1004000001045ED052EA03045BD0C3F30A54C1F383
:100410000A552C44A4F2F3340194A0FB0254C1F316
:10042000130141F48011C3F3130343F4801301FB60
:10043000024400FB034E840A970A44EA815447EAC7
:100440008357A4FB076802958D0A05FB07854FEAD1
:10045000932C04FB0C542705029D4FEA065847EAEB
:100460001637B5EB08056EEB070C870E920E47EAC0
:10047000811742EA8312A7FB0201B6EB0B0164EB82
:1004800000042B0D43EA0C335E1844EB1C50DA4693
:100490005146E7FB0201C5F313044FEA0B3343EA6D
:1004A00014534FEA0432019C43EA0603A4F10C04FE
:1004B0000294009CCDE900B400F01BF903B0BDE844
:1004C000F08F00200146F9E72DE9F04D81EA0304A1
:1004D00004F0004B21F0004514464FF0000A23F0D1
:1004E000004150EA050220D054EA01021DD0C5F3B4
:1004F0000A570246C5F31303C1F31300C1F30A56AA
:1005000040F4801543F48013A7EB0608101BD64671
:1005100008F2FD3873EB050002D308F1010801E091
:1005200092185B41B8F1000F03DA00200146BDE8E4
:10053000F08D00204FF48011064684460EE0171B14
:1005400073EB050705D3121B63EB050306434CEA67
:10055000010C49084FEA300092185B4150EA01074C
:10056000EDD152EA030012D082EA040083EA0501C9
:10057000084305D0101BAB4106D20122002306E040
:1005800000224FF0004302E06FF0010253101AEB1B
:1005900006004CEB085110EB0A0041EB0B01BDE8E3
:1005A000F04D00F097B800F0004230F000400AD063
:1005B000C10D01F56071C0F3160042EA0151C20895
:1005C00040071143704700200146704701F0004387
:1005D00030B421F0004150EA010206D00A0DA2F524
:1005E0006072C1F31301002A02DC30BC00207047A6
:1005F000440F44EAC104C100E01830BC00EBC25013
:1006000000F031B8202A04DB203A00FA02F1002081
:1006100070479140C2F1200320FA03F31943904040
:100620007047202A04DB203A21FA02F000217047AB
:1006300021FA02F3D040C2F120029140084319464A
:100640007047202A06DBCB17203A41FA02F043EA32
:10065000E07306E041FA02F3D040C2F1200291407B
:100660000843194670470029A8BF7047401C49003D
:1006700008BF20F00100704710B4B0FA80FC00FA07
:100680000CF050EA010404BF10BC704749B1CCF132
:10069000200421FA04F411FA0CF118BF01212143BE
:1006A0000843A3EB0C01CB1D4FEA00614FEA102079
:1006B00042BF002010BC704700EBC350104400291B
:1006C000A4BF10BC7047401C490008BF20F00100C7
:1006D00010BC704710B5141E73F1000408DA401CFA
:1006E00041F1000192185B411A4301D120F0010051
:1006F00010BD2DE9F04D92469B4611B1B1FA81F241
:1007000002E0B0FA80F220329046FFF77BFF044609
:100710000F4640EA0A0041EA0B0153465A46084395
:1007200013D0114653EA010019D0C8F140025046D7
:10073000FFF777FF05460E46504659464246FFF7FB
:1007400061FF084305D0012004E020463946BDE89A
:10075000F08D0020054346EAE0762C4337430A98A3
:100760006305E40AA0EB08000022FD0A44EA4754AE
:100770000A3002D500200146E9E701051019694158
:10078000DDE9084500196941BDE8F04DA2E72DE912
:10079000FE4FC3F30A5701F000450024C1F30A5687
:1007A000C3F31303C1F3130143F4801312EB020AE2
:1007B000A64641F48011009543EB030CA7F1010B11
:1007C00016E0B0EB0A0061EB0C01071E71F10007A7
:1007D00007DA4FF00008D0EB080085F0004568EB21
:1007E0000101171A73EB0107EBD3761E001849417C
:1007F0005E45F6DA50EA010209D0CDE900E50022B3
:1008000013460296FFF775FF03B0BDE8F08F204650
:100810000099F9E7064C074D06E0E06840F0010357
:1008200094E8070098471034AC42F6D3FFF7D8FCA1
:1008300080710008A07100080EB5C10F80EAE07059
:100840000844CA07002140F233438DE80E000A46EF
:100850000B46FFF74EFF03B000BD0EB540F233412B
:1008600002910021CDE900110A460B46FFF741FF36
:1008700003B000BD70B5C1F30A5201F00045002479
:10088000C1F3130140F2FF3341F480119A4201DABF
:10089000002070BD40F233439A42A2F2334203DC9F
:1008A0005242FFF7BEFE00E090402C43F1D04042A0
:1008B00070BD000000218161016041608160C16004
:1008C000016101757047000040F22000C2F2000093
:1008D00090ED000A9FED041A9FED042A20EE010A14
:1008E00080EE020A704700BFACFFB33DA34C6542E7
:1008F0004EF2180040F22001CEF20000C2F20001D8
:10090000006891ED000A9FED261A9FED262A20EE41
:10091000010A80EE020A91ED011A9FED232AC860B8
:1009200030EE411AB0EEC13AB4EE423AF1EE10FAAE
:1009300012DDB5EE401A91ED021AB7EE003ABFEEA5
:10094000002AF1EE10FAC8BFB0EE423A33EE011AB7
:1009500081ED021A02E000BF91ED021A9FED132A09
:100960009FED133A21EE021A91ED062A31EE001A9C
:1009700031EE422A82EE032A40F20802C2F200025D
:1009800092ED003A81ED010AB8EEC30A81ED051A35
:1009900081ED061A086122EE000A03F0F3BE00BFE3
:1009A000ACFFB33DA34C65427CD9A040DB0FC940EE
:1009B0006F12833AB0B584B00D4602210DF10E02DC
:1009C0004FF0FF34CDE900216C210C220123029469
:1009D00001F0F2F910B104B0B0BD00BFBDF80E10C7
:1009E000090409BA00EE101AB8EEC00A85ED000A33
:1009F00004B0B0BDFEE7000040F2CC20C2F200001F
:100A000000F07CBD40F22C30C2F2000000F076BD58
:100A100040F28C30C2F2000000F070BD40F2EC30C9
:100A2000C2F2000000F06ABD704700004FF40050B1
:100A300001F01AB8EFF3108072B600BFFEE70000B5
:100A4000B0B52DED048B9FED2C8A40F2040440F2EA
:100A50000805C2F20004C2F20005B0EE080AF0EE8A
:100A6000480A2060296005F09BFB40F6B83000F092
:100A700031FE9FED220AF0EE480A05F091FB28684E
:100A80002168484300EE100AB8EEC09AFFF71CFF39
:100A900040F6B004C2F2000494ED001A29EE000AF8
:100AA00030EE410A10EE100AFFF77DFD41EC100B0D
:100AB0009FED0F1B05F088FD51EC100BFFF786FD35
:100AC00000EE100A30EE081AB5EE400AF1EE10FA08
:100AD000A8BFB0EE401A84ED001AFFF709FF40F2FC
:100AE0001010C2F2000080ED000ABDEC048BB0BD16
:100AF00000000060FB211940DB0FC940000000002E
:100B000040F20C00C2F2000080ED000A04F014BCB8
:100B100070B582B090F85820012A03D1022108460E
:100B200002B070BD002201920092026840F2080CEF
:100B3000C5F2000CB2F1A04F0CF1F80508D040F25C
:100B40000043C5F200039A423ED10CF59F6300E0DA
:100B50002B469B68946823435B0735D44FF4E063CE
:100B6000D1F800E0AA4208BF4FF44073B2F1A04FA1
:100B700008BF4FF440735CF80340BEF1000F24F44B
:100B800060442DD04D6890F838602C4340F2001539
:100B900042F48072C5F2000544EA4634AA424CF899
:100BA000034037D1DCF80020DCF800412243D207B3
:100BB0003AD15CF80320896840F61F74A24341EAE9
:100BC0000E01114322E000BFC16D41F02001C1655B
:100BD0000121002280F85820084602B070BD00BFF5
:100BE00042F4807140F20012C5F2000291424CF8CA
:100BF00003401BD1DCF80010DCF800211143C907C9
:100C00001ED15CF8031040F61F7291434CF803109C
:100C10000021DEE7DCF80044DCF80055DCF80026B3
:100C20002C432243D207C4D00021D2E7DCF80024B1
:100C3000DCF80065DCF8001632431143C907E0D048
:100C40000021C6E7F0B581B00022009290F858204C
:100C5000012A03D10221084601B0F0BD0123076833
:100C600080F85830BB685B0736D4D1E900531F26A3
:100C7000C3F3012407EB8404226B03F01F039E409F
:100C8000B243C5F3846606FA03F31A432263BA68D3
:100C9000BB6802F0040203F00803D21840F0BD80E4
:100CA0000A6807F114030426C2F34064D1F808E08F
:100CB00006EAD25C53F82440C2F304550722AA4046
:100CC000BEF1004F24EA02040CD143F80C401A682C
:100CD00042F000430EE000BFC16D41F02001C1654C
:100CE00001219DE10EFA05F2224343F80C201A6817
:100CF00022F000437B61D1E90435FC68042B5FD10D
:100D00003A6E3A6E0B68C2F3846293FAA3F6C3F3A9
:100D1000846C6FF3DF43B6FA86F5002B2C464FF652
:100D2000FF7E08BF6446A242C0F2070E0CD13A6EA5
:100D300022F000423A660A6802EA0E03C2F3846CAB
:100D400092FAA2F2B2FA82F57A6E7A6E002BC2F3B0
:100D500084622C4608BF6446A2420CD17A6E22F00F
:100D600000427A660A6802EA0E03C2F3846C92FAC1
:100D7000A2F2B2FA82F5BA6EBA6E002BC2F38462A6
:100D80002C4608BF6446A2420CD1BA6E22F0004243
:100D9000BA660A6802EA0E03C2F3846C92FAA2F2FF
:100DA000B2FA82F5FA6EFA6E002BC2F3846208BFC3
:100DB0006546AA4231D1FA6E22F00042FA662CE072
:100DC000062202EA940205FA02FC0E6807F16005A9
:100DD00055F823404FF20002C0F2FF3206F0F84609
:100DE000224046EA0C06324342F0004245F82320F6
:100DF0000A698B6955F8226026F08076334345F8FE
:100E000022300A690B7F55F82260012B26F000760C
:100E100008BF06F1007645F82260BA68D20750D1C3
:100E20000D68CA68D7F8B0602B466FF3DF4326EA37
:100E3000030C4FF6FF7602F01804C0F20706E640F6
:100E400000242E40C4F27F0446EA0C06A242C7F8F2
:100E5000B06036D193B195FAA5F2B2FA82F20132BE
:100E600002F01E03092B02F01F0310D801229A4042
:100E700003EB430342EA035315E000BF012202EBF8
:100E8000956202F01E030A2B02F01F03EED301222B
:100E900000269A4003EB4303CFF6206606EB03538C
:100EA0001A4342F00073C3F3406607EB86068A6874
:100EB0007569C3F3045307249C40A5439A402A4311
:100EC00072610B680021C8F208010B4266D040F243
:100ED000003EC5F2000EAEF500710EF580648F4243
:100EE00004BF40F20034C5F200042146B7F1A04F20
:100EF00004BF40F20031C5F200018D680022CCF23F
:100F00002132934205F0E07C04D01022C9F2C002E5
:100F1000934245D12A0261D440F20062C5F2000238
:100F2000974202D0B7F1A04F5AD18A6822F0E072FE
:100F300042EA0C0242F400028A6040F21801C2F256
:100F40000001096842F663528909C0F23E52A1FBD2
:100F50000212910901EB41010C2202EB8101009187
:100F60000099002948D00099013900910099002981
:100F700044D00099013900910099002940D000998E
:100F800001390091009900293CD000990139009164
:100F9000009900294FF00001E5D141E000213FE038
:100FA0000022CCF25272934208BF15F0807219D021
:100FB0000021CCF684318B424FF0000108BF15F4BC
:100FC00080022DD1B7F1A04F1FD040F20011C5F221
:100FD00000018F4218D1002122E000BF00211FE054
:100FE00000211DE08A6822F0E07242EA0C0242F021
:100FF00080728A60002113E0002111E000210FE0DF
:1010000000210DE000210BE0A646DEF8081021F0DB
:10101000E07141EA0C0141F48001CEF80810002192
:10102000002280F85820084601B0F0BDB0B582B06B
:101030000446002001904CB1E06D58B121688868E9
:10104000800012D48868C00019D54CE0012002B09D
:10105000B0BD00BF204600F027F90020206684F8CC
:101060005800216888688000ECD588684FF6C07207
:10107000C5F6FF72104088608868C00033D44FF610
:10108000C0728868C5F6FF7202F18052104000F10C
:101090008050886040F21800C2F20000006842F6FA
:1010A00063528009C0F23E52A0FB02029009022264
:1010B00002EB400001900198A8B100BF01980138EF
:1010C0000190019878B1019801380190019850B1D0
:1010D000019801380190019828B1019801380190D8
:1010E00001980028EAD18868C00009D4E06D40F07A
:1010F0001000E065206E40F001002066012000E055
:1011000000208A68E36D02F0040203F01003D21895
:10111000E26D40F0818022F481720232E2658A68D9
:10112000D20729D140F2001341F48072C5F20003C6
:1011300040F2080C9A42C5F2000C73D1DCF8003082
:10114000DCF800211A43D20716D10CF1F8024FF453
:10115000E063D4F804E0914208BF4FF44073B1F16A
:10116000A04F08BF4FF440735CF8032022F47C12B8
:1011700042EA0E024CF80320627FE36B43EA4232FC
:10118000D4E902C31A4394F8243042EA0C02012B3A
:1011900042EA034207D1D4F828C00023CFF6FE73F9
:1011A00003EB4C431A43E36A33B103F47873D4F886
:1011B00030C01A4342EA0C02D1F80CC044F20703D3
:1011C000CFF6F07303EA0C031A43CA600A69636B33
:1011D00022F040621A430A618A68120753D494F8D5
:1011E0003820237F520042EA833CCB6844F202025B
:1011F00023EA020242EA0C02CA6022690B69FAB1D0
:1012000043F480330B61D1F8C0C043F6FF732CEA7E
:1012100003031A431CE000BF42F010010120E16506
:1012200002B0B0BDDCF800E4DCF80025DCF80036E4
:1012300042EA0E021A43D2073FF487AF9CE700BF91
:1012400023F480320A61D1F8C02043F6FF739A4339
:10125000C1F8C02094F840300A69012B10D140F247
:10126000FD7322EA030CD4E91132D4E913E543EA11
:101270000C031A4342EA0E022A4342F0010201E043
:1012800022F001020A6162690B6B012A23F00F024E
:1012900002D1236A013B1A430A63E16D012262F322
:1012A0000101E16502B0B0BDF0B59BB0044600207D
:1012B0001A90CDE91800CDE9160001A85421FEF7D7
:1012C000DFFF206840F20041C5F2000188426FD084
:1012D00040F20011C5F20001884200F0A380B0F195
:1012E000A04F40F009814FF4004001904FF00050B2
:1012F000129001A801F040F8002818BFFFF79AFBF0
:1013000040F2EC01C2F200014A6841F24C00C4F222
:101310000200531C4B6042B9016841F40051016066
:10132000016801F4005100910099016816AD41F087
:10133000040101600168032701F004010091009994
:101340000168002641F0010101600068294600F0B3
:101350000100009000980820169040F20040C4F66A
:10136000000000F580601797189600F089FB4FF099
:1013700090402946CDE91677189600F081FB40F29F
:10138000CC250820C2F20005C4F20200052180220B
:101390004FF4007385E8430005F114004FF4006733
:1013A0004FF0200CC5E9036280E888109BE000BF85
:1013B0004FF4803001904FF00040139001A800F0EE
:1013C000DBFF002818BFFFF735FB41F24C00C4F2E9
:1013D00002000168002641F480410160016801F4C7
:1013E000804100910099016841F0020101600068AC
:1013F00016A900F002000090009802201690032029
:10140000179040F20040C4F60000189600F038FB38
:101410000820C4F2020040F28C352830C2F20005E8
:10142000252153E04FF4004001904FF000501290FE
:1014300001A800F0A1FF002818BFFFF7FBFA40F257
:10144000EC01C2F200014A6841F24C00C4F2020011
:10145000531C4B6042B9016841F4005101600168BE
:1014600001F4005100910099016816AD41F00101AD
:1014700001600168032701F00101009100990168F2
:10148000002641F0020101600068294600F00200D8
:1014900000900098C02016904FF090401797189633
:1014A00000F0EEFA0420CDE9160740F20040C4F641
:1014B00000002946189600F0E3FA0820C4F2020062
:1014C00040F22C351430C2F20005242180224FF462
:1014D00000734FF4006728606960AE60EE602A61B7
:1014E0006B61AF61EE6128462E6200F05DF808B1D5
:1014F000FFF7A0FA6565AC621BB0F0BDB0B5D0E9EE
:1015000010C30268DCF8001003F01F030424D2F8B3
:1015100000E09C400C4218BF1EF0040522D10224BA
:101520009C400C4218BF1EF0020529D1D940090782
:1015300024D51EF0080108BFB0BD116821F00E01CE
:101540001160012101FA03F2CCF80420C16380F894
:101550002510416B002280F8242079B1BDE8B0400D
:10156000084700BF1168890603D4116821F00401FF
:101570001160CCF80440016B0029EFD1B0BD00BF71
:101580001168890606D4116821F00A011160012151
:1015900080F82510CCF80440C16A0022002980F8A8
:1015A0002420DBD1EAE7000000284FF0010100F021
:1015B0008E802DE9F04740F2000CC4F2020C036863
:1015C0004FF6F8320CF5816ECBF6FD72734538BFDD
:1015D00002F580624CF6CD441A44CCF6CC44A2FB12
:1015E00004286FF0070252FA83F2A2FB04290CF5DB
:1015F00080656FF00304D0E90262D0F810A03CBF10
:101600000025C4F2020504EA9804C0E9105402253A
:1016100080F825501D6847F6F07725EA070737431D
:101620003A43476942EA0A0285693A43C7692A434D
:10163000056A3A432A431A600CF50262734538BFC3
:101640000CF50062A3180CF50862C264C9F3041219
:1016500040F6840C01FA02F2B6F5804FC4F2020C97
:101660008364026506D1002141601960CCF8002036
:101670001EE000BF41685FFA81FE013903294FF087
:101680000001C3F800E0CCF8002011D8AEF101024F
:101690000CEB820747F87C1F02F01F01012202FABF
:1016A00001F30CF1BC023946CCF8C03002E000BFB7
:1016B0000022002300F1540C8CE80E0000210122CE
:1016C000C16380F8252080F82410BDE8F047084663
:1016D00070470000B0B5044600F0C6FA054640F277
:1016E0001000C2F200004068611C18BF044400BF33
:1016F00000F0BAFA401BA042FAD3B0BD70B5D8B121
:10170000044690F85C0028B9002084F85D0020466B
:1017100000F01EF92068816921F01001816100F05C
:10172000A3FA054620688169090707D500F09CFAED
:10173000401B0B28F6D312E0012070BD816941F0F7
:101740000101816100F090FA054600BF20688169BF
:10175000C9070DD100F088FA401B0B28F6D3206E84
:10176000032140F001002066012084F85C1070BD68
:10177000826946F2004CC4F2000C42F0020260455D
:10178000826102D16268CCF80021227C8369012A3F
:1017900023F0400318BF40338361627C8369012AD0
:1017A00023F4804308BF03F580438361A27C8369EF
:1017B000012A23F4805318BF03F5805383618269A3
:1017C000D4E902E322F4407545EA0E058561856996
:1017D00025F0A4058561056925F0100505619BB11B
:1017E000012B0DD0022B09D08569032B45F0800514
:1017F0008561056945F01005056105D1202300E0EC
:10180000042385692B43836104F114052ACD226AE0
:101810005E1E6FF0FF0303EB052545EA4665013ABE
:101820002A430025CFF6FF7505EB01411143BEF5B4
:10183000407FC16110D1D4E909E2D4E90B61013ADA
:1018400003EB06231A436FF00F0303EB011111435F
:1018500005EB0E421143C160D4E90D13E26BD0F8E1
:10186000C0603243C0F8C0200CF580660CF58042A1
:10187000B04204BF4AF25072C4F200020CF5006696
:10188000B04208BF02F5D4622264D0F8806026F42A
:10189000F81646EA0141C0F8801002F17001616457
:1018A000D0F8801021F0706141EA0361C0F8801027
:1018B00002F1B000A06402F5C470E06402F5187093
:1018C000206502F51E70606502F55470002100BFAE
:1018D000C2E90011C2E90211C2E90411C2E906110C
:1018E000C2E90811C2E90A11C2E90C11C2E90E11DC
:1018F000C2E91011C2E91211C2E91411C2E91611AC
:10190000C2E91811C2E91A11C2E91C11C2E91E117B
:10191000C2E92011C2E92211C2E92411C2E926114B
:10192000C2E92811C2E92A11C2E92C11C2E92E111B
:10193000C2E93011C2E93211C2F8D010D432824269
:10194000C6D300200121A065206684F85C1070BD1C
:1019500010B59CB0044600201B90CDE91900CDE9DC
:10196000170002A85421FEF78BFC206846F6000100
:10197000C4F20001884237D046F20041C4F20001AF
:1019800088426DD14FF4805002904FF0007010905B
:1019900002A800F0F1FC002818BFFFF74BF840F256
:1019A0000C11C2F200010A6841F24C00C4F20200BC
:1019B000531C0B6042B9C16841F00071C160C1683D
:1019C00001F0007101910199016841F0010101608C
:1019D000006800F00100019001984FF4C05017908A
:1019E0004FF0904032E000BF4FF4805002904FF033
:1019F0000070109002A800F0BFFC002818BFFFF78D
:101A000019F840F20C11C2F200010A6841F24C00D0
:101A1000C4F20200531C0B6042B9C16841F000716E
:101A2000C160C16801F0007101910199016841F044
:101A300002010160006800F00200019001984FF47B
:101A40008250179040F20040C4F600000221189125
:101A50000021CDE9191109211B9117A900F010F8F7
:101A60001CB010BD7047000040F21441C4F20101E7
:101A70000A68024214BF08607047FFF7F3BF000016
:101A80002DE9F04F84B08E4641F20042C4F60002C8
:101A9000DEF8004006219042019008BF0521002C8D
:101AA000009100F0D7800198002500F138424FEAFC
:101AB000B2230098012700264FF00008052B38BFFD
:101AC00018460090CDF808E00EE000BFDEF80040B8
:101AD00008F1010834FA07F106F1020607F10107DF
:101AE00005F1040500F0B680A7F1010A012000FA13
:101AF0000AF314EA0309E9D0DEF804C00CF0030B82
:101B0000ABF10104012C17D80198744681680322B7
:101B1000E468B2409143B4402143816041684FEA98
:101B2000480E9943CCF3001303FA0AF30446D0435A
:101B3000194361600CE000BF0321B140019CC84320
:101B4000BBF1030FB64603D1B6464FF0030B23E0BB
:101B5000E168029A01409368BBF1020F03FA0EF3A9
:101B600041EA0301E16017D16FF0030101EA5A0174
:101B7000214405F01C040F23D1F820C003FA04FB14
:101B800013692CEA0B0CA34043EA0C03019C0B6283
:101B9000D2F804C00CF0030B21680BFA0EF20140DE
:101BA00011432160DDF808E01CF4403F8ED041F283
:101BB0006000C4F20200016840F2004C41F00101F3
:101BC00001600168C4F2010C01F001010391039965
:101BD0002AF003014FF6084A6144CFF6FF7A05F078
:101BE0000C030F2051F80A2000FA03F40098A243D6
:101BF00000FA03F31A4341F80A20DCF80810DEF873
:101C0000042041EA090340F20C40D40258BF21EA03
:101C10000903CCF80830C4F201000168940241EADB
:101C2000090358BF21EA09030360DCF80410940398
:101C300041EA090358BF21EA0903CCF80430DCF873
:101C40000010D20341EA090358BF21EA0903CCF886
:101C500000303BE704B0BDE8F08F00001823002AF5
:101C600008BF2823C150704740F6A800C2F2000008
:101C70000068704790F84120202A03D190F8402056
:101C8000012A01D102207047242280F841200268F5
:101C9000136823F001031360136823F48053136067
:101CA000136819431160116841F00101116020218E
:101CB00080F84110002180F840100846704700006D
:101CC00090F84120202A03D190F84020012A01D128
:101CD00002207047242280F841200268136823F014
:101CE00001031360136823F4706343EA0121116058
:101CF000116841F001011160202180F8411000219C
:101D000080F8401008467047002804BF0120704743
:101D100010B5044690F8410028B9002084F840002E
:101D2000204600F065F9242084F8410094E8091069
:101D3000E2680168012A21F00101016023F070616D
:101D40000161816821F40041816003D14CF40041BC
:101D5000816009E04CF40441022A816004D14168A9
:101D600041F4006103E000BF416821F4006141607B
:101D7000416804F1100C41F0007141F400414160F0
:101D8000C16821F40041C1609CE80E10114341EA92
:101D90000321C160216A41EA0C010160016841F040
:101DA0000101016000202021606484F8411020635B
:101DB00084F8420010BD00002DE9F04F81B00446C8
:101DC00090F8410020280DD1DDF828B0BBF1000FBC
:101DD0000CD0DDF82CA0BAF1000F07D094F8400029
:101DE00001280BD1022001B0BDE8F08F4FF4007044
:101DF0006064012001B0BDE8F08F00BF01201D46E6
:101E00001746894684F84000FFF72EFF21680646F2
:101E10008A69120447D422200C9A84F84100402099
:101E20004FF0000884F84200C4F84480C4F824B09D
:101E3000A4F82AA0C4F8348049F6000392464A6800
:101E4000CFF600436FF39F29E8B249EA00401A40F9
:101E5000104400F5005048602046514632469B46EB
:101E600002F046FCA8B9012D08D02068390A816229
:101E700020465146324602F03BFC50B92068F9B288
:101E800081622046402100225346009602F082FBE8
:101E900050B384F84080012001B0BDE8F08F00BF4E
:101EA00088690004B7D520461921324602F0C4FAE9
:101EB00000289ED1FFF7D8FE801B21681A28EFD397
:101EC00088690004ECD5606C40F02000606420203C
:101ED00084F84100002084F8420084F8400001208A
:101EE00001B0BDE8F08F00BF608D40F20008B0F592
:101EF000807FC0F2FF1809D3206808F5105350F80E
:101F0000041F4F4601EA0B02FF210AE0618D2068A1
:101F1000CAB250F8043F49EA024203EA0B0708F547
:101F200092333A431A43FF270BF5806502602185FF
:101F300010E000BF618D2068218550F8042FC9B2E0
:101F400049EA01412A404FF00073114319430160EF
:101F5000608D88B32046042100225346009602F08B
:101F600019FB00287FF445AF2068616A406A087059
:101F7000606A218D01306062481E2085618D0139C3
:101F80006185618D0029E3D00004E1D120468021E4
:101F900000225346009602F0FDFA00287FF429AF94
:101FA000608DB0F5807FC5D32068278550F8041F69
:101FB0004A4629404346C8E720465146324602F089
:101FC00059FB00287FF415AF20682021C1614268C9
:101FD0004EF60003CFF600631A404260002084F8FA
:101FE000411084F8420084F8400001B0BDE8F08F51
:101FF00010B59CB0044600201B90CDE91900CDE936
:10200000170002A85421FEF73BF9206845F60001AD
:10201000C4F20001884237D045F20041C4F2000109
:1020200088425FD14020029002A800F0A5F9002864
:1020300018BFFEF7FFFC41F24C04C4F20204206812
:1020400017A940F002002060206800F00200019013
:1020500001984FF4C0701790122018900020CDE91D
:10206000190004201B9040F20040C4F60000FFF766
:1020700007FDE06840F40010E060E06800F4001044
:10208000019001981CB010BD8020029002A800F0C1
:1020900073F9002818BFFEF7CDFC41F24C04C4F2DE
:1020A0000204206817A940F001002060206800F0B9
:1020B0000100019001984FF4407017901220189081
:1020C0000020CDE9190004201B904FF09040FFF74D
:1020D000D7FCE06840F48000E060E06800F4800035
:1020E000019001981CB010BD40F2100040F6A8010C
:1020F000C2F20000C2F2000140680A6810440860A1
:102100007047000080B5032000F088F8002000F040
:1021100009F800281CBF012080BD00F029F800202C
:1021200080BD000070B540F21006C2F20006716872
:10213000E1B1044640F21800C2F200004FF47A7296
:102140000068B2FBF1F1B0FBF1F000F0CBFE0F2C18
:102150004FF0010508D838B94FF0FF302146002272
:10216000002500F02FF83460284670BD012070BDB6
:1021700082B041F25800C4F20200816841F00101CE
:102180008160816801F0010101910199016841F0CC
:1021900080510160006800F080500090009802B00B
:1021A00000F0E0B8002848BF704700F01F0101228E
:1021B00002FA01F14EF200124009CEF2000242F89A
:1021C0002010704710B54EF60C5CCEF2000CDCF817
:1021D0000030C3F3022E8EF00704042C28BF042421
:1021E000BEF103034FF0FF3E0EFA04F438BF0023A4
:1021F000A14399400EFA03F39A43114300F00F02F2
:10220000043A624409010C3200F16043B0F1FF3F2F
:10221000C8BF03F56442117010BD00004EF60C51AA
:10222000CEF200010A684FF6FF031A4060F30A225B
:1022300042F0806040F0FD7008607047B0F5007FAC
:1022400042D0002840F0808047F21400C4F2000021
:1022500050F8141CC26E01F4C06122F48072B1F512
:10226000806FC2662ED150F8141C012262F34A21FD
:1022700040F8141C40F21801C2F200010968322231
:1022800051434DF68362C4F21B32A1FB0212910C42
:102290000268520511D54A1C0FD0026852050CD5B0
:1022A00059B10268520508D5012906D002685205C5
:1022B00003D50229A1F10401EAD10068400544BF19
:1022C000032070470020704747F21400C4F200005A
:1022D00050F8141CC26E01F4C06142F48072B1F572
:1022E000806FC266EED150F8141C012262F34A21BD
:1022F00040F8141C40F21801C2F2000109683222B1
:1023000051434DF68362C4F21B32A1FB0212910CC1
:102310000268520511D54A1C0FD0026852050CD52F
:1023200059B10268520508D5012906D00268520544
:1023300003D50229A1F10401EAD10068400544BF98
:1023400003207047BEE700BF47F21400C4F200004C
:1023500050F8141C022262F34A2140F8141C002099
:102360007047000047F20800C4F20000016841F421
:1023700080410160704700002DE9F04182B00446C1
:10238000807841F288060007C4F2020602D40020D9
:102390002FE000BF56F8300C10F080580BD156F8E3
:1023A000300C40F0805046F8300C56F8300C00F0FD
:1023B00080500190019847F20007C4F20007386886
:1023C00040F480703860FFF74FFC05463868C00560
:1023D00000F10C81FFF748FC401B0228F6D90320CE
:1023E000B8F1000F05D156F8301C21F0805146F8A5
:1023F000301C2168CA0717D18A071DD44A0723D485
:102400000A0729D4CA062FD48A0635D44A063BD4F3
:102410000A0641D4CA0547D48A034DD48A0553D449
:102420004A0559D467E000BF3268636822F00302AE
:102430001A4332608A07E1D53268A36822F00C02A1
:102440001A4332604A07DBD53268E36822F0300273
:102450001A4332600A07D5D53268236922F0C002D8
:102460001A433260CA06CFD53268636922F44072DB
:102470001A4332608A06C9D53268A36922F44062E1
:102480001A4332604A06C3D53268E36922F44052E7
:102490001A4332600A06BDD53268236A22F44042EC
:1024A0001A433260CA05B7D53268636A22F44032F3
:1024B0001A4332608A03B1D57269A36A22F003021B
:1024C0001A4372618A05ABD53268E36A22F440226E
:1024D0001A4332604A050ED53268236B22F440124B
:1024E0001A43B3F5801F326005D156F87C2C42F4B4
:1024F000801246F87C2C0A050ED53268636B22F4F4
:1025000040021A43B3F5800F326005D156F87C2C97
:1025100042F4801246F87C2CCA040ED53268A36BB4
:1025200022F040721A43B3F1807F326005D156F831
:102530007C2C42F4801246F87C2C8A040ED532683A
:10254000E36B22F040621A43B3F1006F326005D1B1
:1025500056F87C2C42F4801246F87C2C4A040ED5A6
:102560003268236C22F040621A43B3F1006F32608C
:1025700005D156F87C2C42F4801246F87C2C0A04D3
:102580000ED53268636C22F040521A43B3F1805F7B
:10259000326005D156F87C2C42F4803246F87C2C0F
:1025A000CA030ED53268A36C22F040421A43B3F13D
:1025B000804F326005D156F87C2C42F4803246F8C8
:1025C0007C2C49030ED57169E26C21F44011114352
:1025D000B2F5001F716105D156F87C1C41F48011E1
:1025E00046F87C1C02B0BDE8F08100BFB06810F472
:1025F000407010D0216D88420BD0B068B16820F4D3
:10260000407041F48031B160B16821F48031B16033
:10261000B060C0070CD1B068216D20F44070084351
:10262000B0600020B8F1000F7FF4E3AEDBE600BF3E
:10263000FFF71AFB054641F2883700BFB0688007F4
:10264000E9D4FFF711FB401BB842F7D9C7E60000F9
:102650002DE9F04700286DD042F2000AC4F2020AC8
:102660000446DAF800000D4600F00F0088420CD254
:10267000DAF8000020F00F002843CAF80000DAF86A
:10268000000000F00F00A84254D1216841F2080870
:10269000C807C4F2020803D1880740F1D880BDE022
:1026A000606802283AD0032840D158F8082C9201DB
:1026B00040D5D8F80420D8F8043042F2004702F0A0
:1026C0000302C3F30313C0F2F4070133032A04BF68
:1026D00043F20067C0F26E17D8F80420B7FBF3F39B
:1026E000D8F80470C2F306225A43C7F341630227A5
:1026F00007EB4303B2FBF3F24BF20043C0F2C443D7
:102700009A4261D9D8F8002012F0F00F51D0890711
:102710005AD5A168002957D14BE000BF58F8081CD2
:1027200089035CBF0120BDE8F08707E058F8081C6A
:10273000490503D40120BDE8F08700BFD8F8001098
:1027400001F00C0104293FD0D8F8001001F00C0171
:10275000082939D0D8F8001001F00C010C2933D128
:10276000D8F80410D8F8042042F2004301F0030125
:10277000C2F30312C0F2F4030132032904BF43F28F
:102780000063C0F26E13D8F80410B3FBF2F2D8F86D
:102790000430C1F306215143C3F34162022303EB2A
:1027A0004202B1FBF2F14BF20042C0F2C44291424C
:1027B0000AD9D8F80010082262F307114FF0010976
:1027C000C8F8001002E000BF4FF00009D8F8001070
:1027D00021F003010843C8F80000FFF745FA064658
:1027E00041F28837D8F80000616800F00C00B0EBC7
:1027F000810F07D0FFF738FA801BB842F2D90320C7
:10280000BDE8F0872168880708D4B9F1000F1ED011
:10281000D8F8000020F0F00017E000BF480705D509
:10282000D8F8000040F4E060C8F80000080706D5BA
:10283000D8F80000072262F30D20C8F80000D8F88D
:102840000000A26820F0F0001043C8F80000DAF899
:10285000000000F00F00A8421BD9DAF8000020F0B9
:102860000F002843CAF80000FFF7FEF9064641F2C0
:10287000883700BFDAF8000000F00F00A84207D048
:10288000FFF7F2F9801BB842F4D90320BDE8F087C6
:102890002168480707D5D8F80000E26820F4E06016
:1028A0001043C8F80000080708D5D8F800002169CF
:1028B00020F4605040EAC100C8F80000D8F80000D9
:1028C00042F20041C0F2F40100F00C000428084676
:1028D0002DD0D8F8000000F00C00082843F200606A
:1028E000C0F26E1023D0D8F8002002F00C020C2A9F
:1028F0001CD1D8F80420D8F8043002F00302C3F346
:1029000003130133032A08BF0146D8F80400B1FBC2
:10291000F3F1D8F80420C0F306204843C2F3416124
:10292000022202EB4101B0FBF1F000E00020D8F8F8
:10293000001047F23012C1F30311C0F60002515CDF
:1029400040F2180201F01F0120FA01F140F21000DC
:10295000C2F200000068C2F200021160BDE8F04758
:10296000FFF7E0BB40F2180041F20801C2F200009C
:10297000C4F202010068096847F24012C1F3022163
:10298000C0F60002515C01F01F01C8407047000012
:1029900040F2180041F20801C2F20000C4F2020144
:1029A0000068096847F24012C1F3C221C0F6000274
:1029B000515C01F01F01C8407047000041F20C015A
:1029C000C4F2020151F8040C42F20042C0F2F402D7
:1029D00000F00C000428104608BF704751F8040CA2
:1029E00000F00C00082843F20060C0F26E1021D005
:1029F00051F8043C03F00C030C2B1CBF0020704763
:102A0000D1F800C00B680CF0030CC3F303130133BF
:102A1000BCF1030F08BF02460868B2FBF3F2096875
:102A2000C0F306205043C1F34161022202EB410191
:102A3000B0FBF1F0704700002DE9F04182B00028B2
:102A400000F006810446007841F20006C007C4F297
:102A5000020655D12078800774D42078000700F151
:102A600097802078400700F1B7802078800600F139
:102A70000781E569002D00F03082B06800F00C009D
:102A80000C2840F05981012D00F0E280F068216AA5
:102A900000F003028A4240F0DB80626A6FF00F03AD
:102AA00000F0F00103EB0212914240F0D180A16AE4
:102AB00000F4FE42B2EB012F40F0CA80E16A00F060
:102AC0007842B2EBC16F40F0C380226B0023CFF697
:102AD000E07303EB025200F4C0016FF31402914261
:102AE00040F0B680616B4FF07E4202EB016100F076
:102AF000C06001F07E41884240F0AA80EDE100BF55
:102B0000B06800F00C01F06808295BD0032281F066
:102B10000C0122EA00000844B0FA80F0400951D1CB
:102B20006068B0F5803F07D0B0F5A02F40F0DA80A4
:102B3000306840F480203060306840F4803030608D
:102B4000DBE000BFB068F16800F00C00042869D039
:102B500001F0030180F00C0081F002010844B0FA9A
:102B600080F040095ED1E1683068002900F0D28031
:102B700040F480703060FFF777F805463068400514
:102B800000F1FC80FFF770F8401B0228F6D92EE117
:102B90006169D6F89400002900F0908040F00100AF
:102BA000C6F89400FFF760F8054600BFD6F8940019
:102BB00080073FF556AFFFF757F8401B0228F5D9BD
:102BC00015E100BF306880037FF544AF60680028DE
:102BD0007FF440AF3CE000BFB06D10F0805808D1EA
:102BE000B06D40F08050B065B06D00F08050019045
:102BF000019847F20007C4F200073868C0052BD4DB
:102C0000386840F480703860FFF72EF8054600BF42
:102C10003868C00520D4FFF727F8401B0228F7D9F1
:102C2000E5E000BF3068400501D5E06880B170681C
:102C3000216920F0FE4040EA0160706040F210001F
:102C4000C2F200000068FFF76DFA00283FF405AFFC
:102C5000012002B0BDE8F081A068012808D0052855
:102C600040F0AA80D6F8900040F00400C6F890002A
:102C7000D6F8900040F00100C6F89000A9E000BF2F
:102C8000A169D6F89800002900F0808040F001008A
:102C9000C6F89800FEF7E8FF054600BFD6F8980092
:102CA00080073FF5E6AEFEF7DFFF401B02284FF03E
:102CB0000300F3D902B0BDE8F08100BF20F00100AD
:102CC000C6F89400FEF7D0FF054600BFD6F8940082
:102CD00080077FF5C6AEFEF7C7FF401B0228F5D977
:102CE00085E000BF3168002821F48031316031680F
:102CF00021F48021316000F07F80FEF7B5FF0546AA
:102D0000306880033FF5A6AEFEF7AEFF401B642897
:102D1000F6D96CE020F480703060FEF7A5FF054620
:102D2000306840057FF599AEFEF79EFF401B0228F4
:102D30004FF00300F4D9BDE7306820F080703060B8
:102D4000FEF792FF022D05460CD100BF30688001CE
:102D500040F17E80FEF788FF401B02284FF0030001
:102D6000F4D9A7E73068800140F1B080FEF77CFF1E
:102D7000401B02284FF00300F4D99BE770682169DB
:102D800020F0FE4040EA0160706066E620F001003D
:102D9000C6F89800FEF768FF054600BFD6F8980011
:102DA00080077FF566AEFEF75FFF401B02284FF0FD
:102DB0000300F3D97EE700BFD6F8901021F001019F
:102DC000C6F89010D6F8901021F00401C6F89010C3
:102DD00010B3FEF749FF054641F28837D6F8900058
:102DE00080072BD4FEF740FF401BB842F6D90320E2
:102DF00002B0BDE8F08100BFFEF736FF054600BF18
:102E0000306880037FF526AEFEF72EFF401B642856
:102E10004FF00300F4D94DE7FEF726FF054641F2D7
:102E2000883700BFD6F89000800707D5FEF71CFF53
:102E3000401BB8424FF00300F4D93BE7B8F1000F54
:102E40007FF413AEB06D20F08050B0650DE600BF8A
:102E5000F06848F20C01C0F29F1104F1200700EA6B
:102E6000010C8ECF6FF00F00D4E90C5400EB021070
:102E70000022CFF6E07241EA0C0102EB0552084352
:102E80006FF314024FF07E4540EA032005EB046522
:102E9000104305F07E4540EAC7602843F060306883
:102EA00040F080703060F06840F08070F060FEF7B5
:102EB000DBFE0446306880010FD4FEF7D5FE001B10
:102EC00002284FF00300F5D9F4E600BFF0684FF692
:102ED000FC71CFF6EE610840F060002002B0BDE862
:102EE000F0810000411E0020B0EB116F1CBF0120DB
:102EF00070474EF21002CEF2000251604EF623519E
:102F0000CEF20001F0230B70072190601160704732
:102F1000704700007047000070470000B0B590F89F
:102F20003C20012A04BF0220B0BDD1E90232D1E920
:102F300000CE22F47C5223F4705343EA020448F298
:102F4000FF73CEF6F0730EEA0302224303F500642A
:102F500004EA0C0442EA040C0C6903F5C052224056
:102F60004C6942EA0C02224303F5605422400C6B88
:102F700003F5F04323401A438B6940F2000CCC69FF
:102F8000CEF6FF7C0CEA034C1443026842F6004381
:102F9000C4F201039A4244EA0C030BD045F2000448
:102FA000C4F20104A24205D043F20044C4F2010479
:102FB000A24217D14FF6FF74CDF60F4403EA040E78
:102FC000D1E9084CD1E90A310025CDF6F04505EAF2
:102FD000035343EA0E0324F008552B432CF000550D
:102FE0002B430B430021536480F83C100846B0BDCE
:102FF000B0B5044690F83C00012804BF0220B0BDE3
:103000000D462068D1E90021AB684FF0010C84F82F
:103010003CC002F051FB2068816DD5E9042321F00A
:10302000E7012D7B19431143012D08BF41F0200119
:1030300041F001018165002084F83C00B0BD000032
:10304000704700000168886D40F0010200208A6529
:1030500070470000704700007047000070B590F89E
:103060003C20012A4FF0020265D080F83D20026822
:1030700042F600435468D2F808C0C4F2010345F296
:10308000000E9A42C4F2010E18BF72452CD14D6851
:1030900024F470042C434FF68F75CFF6FF550E685D
:1030A0002C4042F6FF35C4F201053443AA42546075
:1030B0000EDC40F2FF73C4F200039A421CDCB2F152
:1030C000804F2DD040F20043C4F2000326E000BF41
:1030D00043F6FF74C4F20104A24219DC9A421FD0E5
:1030E00043F2004318E000BF43F20045C4F201057B
:1030F000AA42CCD0CFE700BF40F60003C4F20003E1
:103100009A420DD040F60043C4F2000306E000BF2F
:10311000724505D044F20003C4F201039A4204D17F
:1031200089682CF08003194391600121002280F806
:103130003D1080F83C20104670BD000041B10829C8
:1031400010D0042914BF00F1470200F145020BE042
:1031500090F84420012A1CBF01207047022280F809
:10316000442013E000F146021278012A1CBF01201E
:1031700070470222082907D0042914BF80F847208D
:1031800080F8452002E000BF80F84620026801F088
:103190000F000421136A01FA00F023EA0001116212
:1031A000116A08431062506C42F6FF31C4F201010B
:1031B00040F400408A4250640EDC40F2FF70C4F2DA
:1031C0000000824218DCB2F1804F2DD040F2004066
:1031D000C4F2000026E000BF43F6FF70C4F2010015
:1031E000824215DC42F60040C4F2010082421BD04C
:1031F00043F2004014E000BF40F60000C4F20000BB
:10320000824211D040F60040C4F200000AE000BF44
:1032100045F20000C4F20100824205D044F20000F1
:10322000C4F2010082420CD190680721C0F2010172
:10323000014006294FF0000008D0B1F5803F08BFDB
:103240007047106840F001001060002070470000D7
:1032500070470000002804BF0120704710B50446E5
:1032600090F83D0028B9002084F83C00204600F08A
:1032700023F8022084F83D002068211D02F076F931
:10328000012084F8480084F83E0084F83F0084F868
:10329000400084F8410084F8420084F8430084F838
:1032A000440084F8450084F8460084F8470084F818
:1032B0003D00002010BD000082B0006843F20041D4
:1032C000C4F20101884215D042F60041C4F2010166
:1032D00088421CD141F26000C4F20200016841F44E
:1032E00000610160006800F400600190019802B084
:1032F000704700BF41F26000C4F20200016841F46F
:1033000000510160006800F400500090009802B085
:103310007047000080B590F83C20012A4FF002026F
:1033200000F0988080F83D20D0F800C08822DCF8BA
:103330000830CFF6CE721A40CCF808200B68B3F5EF
:10334000005F0DDA3F2B21DD5F2B33DD602B00F0BA
:103350008380702B00F0A280B3F5805F73D0E7E02C
:103360002F22C0F21002934218DD4F21C0F210014B
:103370008B4247DD5021C0F210018B4257D06021B3
:10338000C0F210018B4252D070214BE01F2B41DC68
:10339000002B4CD0102B4AD0CAE000BFB3F1101F55
:1033A0003EDAB3F5005F00F08D80B3F5801F3ED0AC
:1033B000BEE000BF402B00F09980502B40F0B88059
:1033C000D1F804E0C968DCF82030DCF8202022F0D5
:1033D0000102CCF82020DCF8182022F0F00242EAAA
:1033E000011123F00A0242EA0E02CCF81810CCF8C0
:1033F0002020DCF808104FF68872CFF6CF7211400B
:1034000057311EE03021C0F210018B420FD0402115
:1034100008E000BF202B0AD0302B08D088E000BF86
:1034200005D02021C0F210018B4240F08180DCF8F1
:1034300008104FF68872CFF6CF721140194341F051
:103440000701CCF808100022012180F83D1000216E
:1034500080F83C10104680BDD1F804E0C968DCF863
:103460002030DCF8202022F01002CCF82020DCF8FC
:10347000182022F4704242EA013123F0A00242EA0D
:103480000E12CCF81810CCF82020DCF808104FF6FB
:103490008872CFF6CF7211406731D2E7D1E901E3EC
:1034A000C968DCF8082043EA0E0322F47F4243EAAD
:1034B00001211143CCF80810DCF8081041F0770125
:1034C000BFE700BFD1E901E3C968DCF8082043EA9F
:1034D0000E0322F47F4243EA01211143CCF8081085
:1034E000DCF8081041F48041ABE700BFD1F804E0FC
:1034F000C968DCF82030DCF8202022F00102CCF88A
:103500002020DCF8182022F0F00242EA011123F01A
:103510000A0242EA0E02CCF81810CCF82020DCF89F
:1035200008104FF68872CFF6CF721140473188E706
:10353000012289E7002804BF012070472DE9F047E8
:10354000044690F83D000D4628B9002084F83C0060
:10355000204600F04BF8022084F83D0020684BF62E
:10356000F8728168CFF6FE7211408160211D01F072
:10357000FDFF20684FF6FF7881688269D0F820C08F
:10358000D5E9003ED5E9026A43EA0109AB6922EABE
:10359000080246EA03234FF6FC46B343D5E9076722
:1035A00042EA0A0229691A4342EA062242EA011162
:1035B0002CF0AA026B6942EA0E0241EA073142EAA4
:1035C0000312C0F8089081610262012084F848006B
:1035D00084F83E0084F83F0084F8440084F84500F5
:1035E00084F83D000020BDE8F08700002DE9F0419F
:1035F00086B0006840F20041C4F200010026884213
:10360000CDE90466CDE90266019649D0B0F1804F5C
:1036100040F09E8041F24C00C4F20200C1680DF1FE
:10362000040841F00101C160C168022601F00101F6
:10363000009100990168002741F0010101600168D3
:103640004FF0904401F0010100910099016841F0B0
:10365000020101600068414600F0020000900098FD
:10366000202001904FF090400296CDE90377059617
:10367000FEF706FA4FF4816001A9C1C140F2004093
:103680000125C4F60000414604970595FEF7F8F9B8
:103690004FF4004001A9C1C1CDE904751C254BE0E0
:1036A00041F24C00C4F20200C16801AC41F00201D9
:1036B000C160C168022701F0020100910099016810
:1036C00041F001010160016801F0010100910099E0
:1036D000016841F002010160016801F002010091FE
:1036E0000099016841F0080101600068214600F07E
:1036F000080000900098102001904FF09040CDE914
:103700000276CDE90467FEF7BBF940F200451120CF
:10371000C4F60005CDE9010728462146CDE9036638
:103720000597FEF7ADF9042005F500641D25CDE9E8
:103730000107CDE90366059701A92046FEF7A0F928
:10374000284600210022FEF73DFD2846FEF72AFD0F
:1037500006B0BDE8F081000080B590F83E2090F8FA
:103760003F3090F844E090F845C004290AD0B9B938
:10377000012A4FF0010208BFBEF1010F34D01046FC
:1037800080BD00BF012B4FF0010208BFBCF1010F4B
:10379000F5D1022180F83F1080F8451000681EE046
:1037A000012A4FF0010208BF012BE8D1BEF1010F41
:1037B000E5D1BCF1010FE2D1022280F83E2080F871
:1037C0003F2080F8442080F8452091B10068016ACC
:1037D00021F001010162016A41F001010162102141
:1037E0006FF0100209E000BF022180F83E1080F85F
:1037F0004410006801216FF00102036A1A4002625E
:10380000026A114301620168002241F00101016076
:10381000104680BD70470000F0B581B004460068D6
:10382000C5680669B10717D515F0020114D06FF00D
:1038300002010161012121778069800704D02046BF
:10384000FFF7E8FF06E000BF204600F03BF9204606
:1038500000F06EFB00202077700719D515F00400EA
:1038600016D020686FF00401016102212177806980
:1038700010F4407F04D02046FFF7CCFF06E000BFE5
:10388000204600F01FF9204600F052FB0020207770
:10389000300717D515F0080014D020686FF0080124
:1038A000016104212177C069800703D02046FFF71A
:1038B000B1FF05E0204600F005F9204600F038FB96
:1038C00000202077F00619D515F0100016D02068DA
:1038D0006FF01001016108212177C06910F4407F69
:1038E00004D02046FFF796FF06E000BF204600F018
:1038F000E9F8204600F01CFB00202077F00718BFF5
:1039000015F0010006D020686FF00101016120462A
:1039100000F0E0FB16F4025F05F0800718BF002FEF
:1039200002D1F00509D410E020686FF40251016162
:103930002046FFF7EFFAF00507D537B120686FF49E
:10394000807101612046FFF7E3FA700609D515F092
:10395000400006D020686FF040010161204600F071
:10396000BBFBB00609D515F0200006D020686FF02B
:10397000200101612046FFF7CFFAF00209D515F4C6
:10398000801006D020686FF4801101612046FFF797
:1039900061FBB00209D515F4001006D020686FF461
:1039A000001101612046FFF74BFB700209D515F4A9
:1039B000800006D020686FF4800101612046FFF787
:1039C0004BFB30020CD515F4000009D021686FF4D0
:1039D000000220460A6101B0BDE8F040FFF738BCA4
:1039E00001B0F0BDF0B587B0006843F20042C4F208
:1039F000010200219042CDE90511CDE903110291A8
:103A00003ED042F60041C4F20101884258D141F251
:103A10004C00C4F20200016840F2004441F004018D
:103A200001600168C4F6000401F0040101910199EC
:103A3000016802AD41F0020101600068022600F059
:103A400002000190019807200290002704F5806091
:103A500029460396CDE904770696FEF711F84FF450
:103A6000C04002A9C1C106200690204629460597FC
:103A7000FEF706F84FF4004002A9C1C1059719E00E
:103A800041F24C00C4F20200026842F004020260FB
:103A9000006800F00400019001984FF4EE5002908D
:103AA0000220CDE9030140F20040C4F6000000F519
:103AB000806405910420069002A92046FDF7E0FFEE
:103AC00007B0F0BD704700002DE9F04190F83C30A0
:103AD000012B04BF0220BDE8F0814FEAB202052AA3
:103AE00000F2A281DFE812F006005400AE000801E7
:103AF0006201A80103681D6A1A6AA3F1804622F0D8
:103B000001021A621A46D3F8048052F818EF8F683F
:103B1000A6F59636D1F800C025F002054FEAB62684
:103B2000092E45EA07050BD80127B74040F2E524E6
:103B300027421FBFCC6825F00C0524F00404254360
:103B4000092E0CD80124B44040F2E52634421FBFB0
:103B500028F44074D1E90567344344EA07084FF676
:103B60008C74CFF6FE740EEA040747EA0C07C3F81C
:103B700004809F614F6809695F631D629F6947F018
:103B800008079F619F6927F004079F6192E100BFCA
:103B9000036842F600461D6A1A6AC4F2010622F062
:103BA00010021A621A465C6852F818EFB3428E6827
:103BB000D1F800C025F0200545EA06150BD045F2E6
:103BC0000006C4F20106B34205D043F20046C4F237
:103BD0000106B34207D1CE686FF0400725F0C0055B
:103BE00007EA06163543A3F18046A6F596364FEA56
:103BF000B626092E0ED8012707FA06F640F2E52769
:103C00003E421FBF24F44064D1E9056744EA8604BC
:103C100044EA870448F6FF46CFF6FF660EEA060739
:103C200047EA0C275C609F614F6809699F631D62CA
:103C30009F6947F400679F619F6927F480679F61D0
:103C400037E100BF036842F600461D6A1A6AC4F2F3
:103C5000010622F480721A621A465C6852F81CCF80
:103C6000B3428E68D1F800E025F4007545EA0625D8
:103C70000BD045F20006C4F20106B34205D043F270
:103C80000046C4F20106B34207D1CE6840F2FF47B6
:103C9000360225F44065BE433543A3F18046A6F5C0
:103CA00096364FEAB626092E0ED8012707FA06F6F1
:103CB00040F2E5273E421FBF24F44054D1E9056796
:103CC00044EA061444EA07144FF68C76CFF6FE76E3
:103CD0000CEA060747EA0E075C60DF614F68096976
:103CE000DF631D62DF6947F00807DF61DF6927F0E6
:103CF0000407DF61DEE000BF036842F600461D6A8C
:103D00001A6AC4F2010622F480521A621A465C68EA
:103D100052F81CCFB3428E68D1F800E025F400556C
:103D200045EA06350BD045F20006C4F20106B3425F
:103D300005D043F20046C4F20106B34207D1CE6873
:103D400044F6FF77360325F44045BE433543A3F1DF
:103D50008046A6F596364FEAB626092E0ED80127DC
:103D600007FA06F640F2E5273E421FBF24F440441E
:103D7000D1E9056744EA861444EA871448F6FF4609
:103D8000CFF6FF660CEA060747EA0E275C60DF61A4
:103D90004F6809691F641D62DF6947F40067DF61CE
:103DA000DF6927F48067DF6183E000BF0368D3F831
:103DB00020C01A6AA3F1804722F480321A621A46A0
:103DC000A7F596375D6852F8508FD1F800E08E68FD
:103DD0004FEAB727092F0AD80124BC4040F2E52753
:103DE0003C421EBF4C6925F4803545EA04252CF47D
:103DF000003747EA06474FF68C76CFF6FE76033655
:103E000006EA080646EA0E065D601E654E68096908
:103E10009E641F621F6D47F008071F651F6D27F026
:103E200004071F6546E000BF0121002280F83C2006
:103E30000846BDE8F08100BF0368D3F820C01A6AC5
:103E4000A3F1804722F480121A621A46A7F596372A
:103E50005D6852F8508FD1F800E08E684FEAB727BE
:103E6000092F0AD80124BC4040F2E5273C421EBF7E
:103E70004C6925F4802545EA84252CF4001747EA8F
:103E8000065748F6FF46CFF6FF6606F5407606EA87
:103E9000080646EA0E265D601E654E680969DE6406
:103EA0001F621F6D47F400671F651F6D27F4806751
:103EB0001F6509021368194311600021002280F870
:103EC0003C200846BDE8F081002804BF012070476F
:103ED00010B5044690F83D0028B9002084F83C0055
:103EE000204600F023F8022084F83D002068211DC0
:103EF00001F03CFB012084F8480084F83E0084F87F
:103F00003F0084F8400084F8410084F8420084F8BF
:103F1000430084F8440084F8450084F8460084F89F
:103F2000470084F83D00002010BD000070470000ED
:103F30007047000061B10A1F4FEAB202032A15D888
:103F4000DFE802F00218101C00F13F0318E000BF88
:103F500090F83E20012A1CBF01207047022280F801
:103F60003E202CE000F141030AE000BF00F14303D2
:103F700006E000BF00F1400302E000BF00F1420391
:103F80001B78012B1CBF01207047032A0CD8DFE8E7
:103F900002F0030F071300BF022280F83F200EE05B
:103FA000022280F841200AE0022280F8432006E045
:103FB000022280F8402002E0022280F842200268BB
:103FC00001F01F010120136A00FA01F18B43136213
:103FD000136A0B43A2F18041A1F596314FEAB1215A
:103FE0000729136258D8884010F0E50F54D0506C60
:103FF00042F6FF31C4F2010140F400408A425064AD
:104000000EDC40F2FF70C4F20000824218DCB2F114
:10401000804F2DD040F20040C4F2000026E000BFE7
:1040200043F6FF70C4F20100824215DC42F6004004
:10403000C4F2010082421BD043F2004014E000BFF2
:1040400040F60000C4F20000824211D040F6004069
:10405000C4F200000AE000BF45F20000C4F2010013
:10406000824205D044F20000C4F2010082420CD129
:1040700090680721C0F20101014006294FF00000BD
:1040800008D0B1F5803F08BF7047106840F00100CC
:1040900010600020704700BF42F6FF30C4F20100FC
:1040A0008242AEDD43F6FF70C4F201008242BDDD04
:1040B00044F20000C4F201008242D9D045F200006F
:1040C000C4F201008242E0D1506C40F400405064E0
:1040D000CEE70000704700007047000090F88410A1
:1040E000012904BF022070472421C0F8881002680B
:1040F0001168136823F00103136021F000530021BD
:10410000416613602022C0F8882080F88410084699
:1041100070470000B0B590F88420012A04BF022047
:10412000B0BD2422C0F888200268D0F864E0D2F83C
:1041300000C01368BEF1000F23F001031360936801
:1041400023F0606341EA0301916019D0936891689C
:1041500047F2701E490FC0F6000E47F278151EF8A0
:104160000140C0F60005695CC3F34263E400B4FBA0
:10417000F1F11EF80340EB5CE500B5FBF3F301E061
:1041800001210123A0F86A102021A0F86830C2F8AC
:1041900000C0C0F88810002180F884100846B0BD27
:1041A000B0B590F88420012A04BF0220B0BD2422BB
:1041B000C0F888200268D0F864E0D2F800C0136824
:1041C000BEF1000F23F001031360936823F06043F6
:1041D00041EA0301916019D09368916847F2701E1B
:1041E000490FC0F6000E47F278151EF80140C0F6E0
:1041F0000005695CC3F34263E400B4FBF1F11EF80F
:104200000340EB5CE500B5FBF3F301E00121012382
:10421000A0F86A102021A0F86830C2F800C0C0F8E9
:104220008810002180F884100846B0BD10B5D8B1C0
:104230000446D0F8880028B9002084F8840020467D
:1042400000F026F82420C4F888002068A16A0268DB
:1042500022F00102026011B1204601F039FA204635
:1042600001F062FB012801D1012010BD21684868DE
:1042700020F490404860886820F02A008860086830
:1042800040F0010220460A60BDE8104001F094BAF7
:1042900070B59CB0044600201B90CDE91900CDE913
:1042A000170002A85421FBF7EBFF206844F6000139
:1042B000C4F20001884239D043F60001C4F2010182
:1042C000884265D048F20001C4F2000188425DD105
:1042D0002020029002A8FEF74FF8002818BFFCF734
:1042E000A9FB41F24C00C4F20200016941F0010156
:1042F0000161016901F0010101910199016841F039
:10430000010101600068022100F0010001900198A4
:104310000C20189100211790CDE919111B9017A9B5
:104320004FF09040FDF7ACFB1CB070BD0420029034
:1043300002A8FEF721F8002818BFFCF77BFB41F22A
:104340004C00C4F20200C16841F48021C160C16820
:1043500001F4802101910199016841F0020101609D
:10436000006817A900F00200019001984FF4206046
:104370001790022018900020CDE9190007201B900B
:1043800040F20040C4F60000FDF77AFB1CB070BD9F
:104390000120029002A8FDF7EFFF002818BFFCF7EC
:1043A00049FB41F24C00C4F202004169002641F48D
:1043B00080414161416901F48041019101990168A5
:1043C00041F004010160006817A900F004000190A9
:1043D0000198302017900220189007201B9040F27F
:1043E0000040C4F6000000F58060CDE91966FDF7D5
:1043F00047FB40F2EC354420C2F20005C4F2020053
:104400001921102285E847004FF4805080234FF097
:10441000200C28622846C5E90436C5E9066CFDF77C
:10442000C3F8002818BFFCF705FBE567AC621CB0B9
:1044300070BD0000FEE7000070B504460068154638
:104440008369DA0602D40021002266E00E461021BC
:10445000C161816989065CD4711C50D036BBFDF7FF
:1044600003FC2068426894F8421083691B040BD552
:1044700012F4804208D1202906D0416841F48041DD
:104480004160FDF7F1FB054620688169890605D486
:10449000FDF7EAFB401B1A28F6D328E0816989065C
:1044A000DDD536E020688169890632D4FDF7DCFB72
:1044B000401BB042F6D92068426894F842108369E4
:1044C0001B040BD512F4804208D1202906D0416884
:1044D00041F480414160FDF7C7FB054620688069D3
:1044E0008006DFD4FDF7C0FB401B1A28F6D32068F6
:1044F00001228169242110E08169890609D481693A
:10450000890606D4816989065CBF81695FEA816199
:10451000F2D52021C161012204218369DE0505D580
:104520004FF4807241F00101C26101225E0505D4A1
:104530009B050AD472B9002070BD00BF41F008018C
:104540004FF480629B05C26104D541F002014FF433
:104550000072C2618269920744BF0022826282694E
:10456000D20703D1826942F00102826142684EF6AD
:104570000003CFF600631A404260606C0843606439
:10458000202084F84100002084F8420084F8400094
:10459000012070BD2DE9F0410446006880690840A3
:1045A000401AB0FA80F04009904233D1DDF818800B
:1045B00015460E461F46581C1CD0BFBB2046002186
:1045C0004246FFF739FF002851D1FDF74DFB206827
:1045D00081693140891BB1FA81F14909A9423AD078
:1045E00080693040801BB0FA80F04009A842E5D0D5
:1045F00010E000BF20464FF0FF314246FFF71CFF9E
:10460000A8BB206880693040801BB0FA80F0400968
:10461000A842EFD00020BDE8F08100BF80693040A3
:10462000801BB0FA80F04009A842F3D120463946F9
:104630004246FFF701FFD0B9FDF716FBA0EB0801DA
:104640002068B942EAD981693140891BB1FA81F108
:104650004909A942E2D1606C40F02000606420204A
:1046600084F84100002084F8420084F840000120D2
:10467000BDE8F08170B5044600688069800635D4D5
:1046800015460E4619B928E0806980062ED42046CA
:1046900031462A46FFF7D0FE30BBFDF7E5FA411B55
:1046A0002068B142F0D981698906EDD4606C40F090
:1046B00020006064202084F84100002084F842003B
:1046C00084F84000012070BDFDF7CEFA20688169B2
:1046D0008906EBD58069800608D4204600212A4649
:1046E000FFF7AAFE0028EFD0012070BD002070BDAA
:1046F00070B5044600688069800720D415460E46D0
:10470000481C11D00EBB00BF204600212A46FFF7EF
:1047100093FEA8BBFDF7A8FA20688169890723D515
:1047200080698007F0D50AE020464FF0FF312A4625
:10473000FFF782FE20BB206880698007F4D5002047
:1047400070BD00BF80698007F9D4204631462A46F3
:10475000FFF772FEA0B9FDF787FA411B2068B1424E
:10476000F0D981698907EDD4606C40F02000606465
:10477000202084F84100002084F8420084F84000A2
:10478000012070BD40F6AC00C2F2000090ED001AAE
:104790009FED062A9FED063A20EE020A21EE031A4B
:1047A00031EE000A80ED000A704700BFCDCCCC3D51
:1047B0006666663F10B58CB040F28810C2F2000009
:1047C0004FF0A04100244FF4403201234FF0040C7D
:1047D00080E8160003210B94CDE90944CDE9074494
:1047E000CDE90544CDE90344CDE90144C0E90344E2
:1047F000C0E9053C8483016280F82430C0E90A34B2
:10480000046380F83840C46380F84040FCF70EFC35
:10481000002818BFFCF70EF940F28810C2F2000021
:1048200009A90994FCF774F9002818BFFCF702F9EC
:104830000220C0F23040019006207F21029000202B
:10484000049104210390CDE9051040F28810C2F2D2
:10485000000001A9FCF7F6F9002818BFFCF7EAF8F8
:104860000420C0F6600001900C20029040F28810F5
:10487000C2F2000001A9FCF7E5F9002818BFFCF717
:10488000D9F840F20020C2F2B050019012200290FC
:1048900040F28810C2F2000001A9FCF7D3F9002809
:1048A00018BFFCF7C7F80CB010BD0000B0B588B059
:1048B00040F2F41040F20011C2F20000C5F2000113
:1048C00000244FF440320123042580E81600032120
:1048D000CDE90644CDE90444CDE90244CDE90044E4
:1048E000C0E90344C0E905358483016280F82430BF
:1048F000C0E90A34046380F83840C46380F840405B
:10490000FCF794FB002818BFFCF794F80820C0F6C9
:10491000904000900620CDE901047F20CDE90305F9
:1049200040F2F410C2F2000069460594FCF78AF9DF
:10493000002818BFFCF77EF81020C1F2C0000090DC
:104940000C20019040F2F410C2F200006946FCF71E
:1049500079F9002818BFFCF76DF841F20000C3F2A6
:10496000602000901220019040F2F410C2F200008A
:104970006946FCF767F9002818BFFCF75BF808B038
:10498000B0BD000010B58CB040F2602040F2004194
:10499000C2F20000C5F2000100244FF4403280E86A
:1049A00016004FF48071042381830121CDE90A446C
:1049B000CDE90744CDE90544CDE90344CDE90144FF
:1049C000C0E90344C0E90543016280F82440C0E91E
:1049D0000B4480F83840C46380F84040FCF726FB65
:1049E000002818BFFCF726F840F26020C2F2000051
:1049F00009A90994FCF78CF8002818BFFCF71AF8ED
:104A00000220C0F23040019006207F210290002059
:104A1000049104210390CDE9051040F26020C2F218
:104A2000000001A9FCF70EF9002818BFFCF702F8F6
:104A30000CB010BD80B582B041F24800C4F2020053
:104A40000168002241F004010160016801F00401E5
:104A500001910199016841F00101016000680021A4
:104A600000F00100009000980B20FDF7ABFB0B203D
:104A7000FDF798FB0C2000210022FDF7A3FB0C2082
:104A8000FDF790FB0D2000210022FDF79BFB0D2080
:104A9000FDF788FB0E2000210022FDF793FB0E207E
:104AA00002B0BDE88040FDF77DBB000080B540F25C
:104AB0004C4046F20041C2F20000C4F20001002264
:104AC000C0E900124FF0100C01230221C0E90222BC
:104AD000C0F80F20C0E905C3C0E90711C0E90933D8
:104AE000C0E90B33C0E90D22C263FCF707FE0028C2
:104AF00008BF80BDBDE88040FBF79CBF80B540F299
:104B0000B04046F60001C2F20000C4F200010022EB
:104B1000C0E900124FF0100C01230221C0E902226B
:104B2000C0F80F20C0E905C3C0E90711C0E9093387
:104B3000C0E90B33C0E90D22C263FCF7DFFD00289A
:104B400008BF80BDBDE88040FBF774BF2DE9F04190
:104B500086B0002641F24C00CDE90466C4F20200A2
:104B6000016840F6000441F0040101600168C4F6E8
:104B7000000401F00401009100990168002241F055
:104B80002001016001684FF4007701F020010091DD
:104B90000099016841F001010160016801F0010123
:104BA00000910099016841F002010160016801F083
:104BB000020100910099016841F00801016000685C
:104BC0004FF4007100F00800009000982046FDF7B7
:104BD00045F84FF090404FF4806100224FF4806818
:104BE000FDF73CF84FF4005001904FF4881001ADF0
:104BF000CDE9020620462946FCF742FF019701272E
:104C000020462946CDE902760496FCF739FF4FF09D
:104C100090402946CDE90187CDE90366FCF730FFD6
:104C2000282000210022FDF7CDFA2820FDF7BAFA4E
:104C300006B0BDE8F081000080B540F2145045F2A6
:104C40000041C2F20000C4F2000142F69B52002370
:104C5000C1F280024FF0010C80E80E10C0E904336D
:104C6000C0E906330362FDF74FF8002818BFFBF7D1
:104C7000E1FE40F21450C2F200000021FCF7FAFFFE
:104C8000002818BFFBF7D6FE40F21450C2F2000015
:104C90000021FDF715F8002808BF80BDBDE8804061
:104CA000FBF7C8BE80B540F2685045F60001C2F27D
:104CB0000000C4F200014AF2FB720023C3F2A0021A
:104CC0004FF0010C80E80E10C0E90433C0E9063350
:104CD0000362FDF719F8002818BFFBF7ABFE40F29E
:104CE0006850C2F200000021FCF7C4FF002818BF82
:104CF000FBF7A0FE40F26850C2F200000021FCF772
:104D0000DFFF002808BF80BDBDE88040FBF792BEF2
:104D100080B540F2BC5048F20001C2F20000C4F27B
:104D2000000143F2243200234FF00C0CC0F20302C6
:104D300080E80E00C0E90333C0E905C3C0E90833C9
:104D40008362FFF773FA002818BFFBF773FE40F287
:104D5000BC50C2F200000021FFF722FA002818BF61
:104D6000FBF768FE40F2BC50C2F200000021FFF7E2
:104D7000D1F9002818BFFBF75DFE40F2BC50C2F22B
:104D80000000FFF7ABF9002808BF80BDBDE88040F8
:104D9000FBF750BE10B59CB0002401A834211B9431
:104DA000CDE91944CDE91644CDE91444CDE91244C6
:104DB000CDE91044CDE90E44FBF762FA40F25060B1
:104DC00042F60041C2F20000C4F2010141F27B52FE
:104DD000C0E90014C0E90242C0E904448461FEF75E
:104DE00039FA002818BFFBF725FE4FF480501890C1
:104DF00040F25060C2F2000018A9FEF78BFA0028BA
:104E000018BFFBF717FE40F25060C2F20000FFF738
:104E10005BF8002818BFFBF70DFE40F2506000243D
:104E2000C2F2000015A9CDE915441794FEF716F952
:104E3000002818BFFBF7FEFD6020CDE90E0440F20C
:104E40005060C2F200000EA90022CDE91044CDE965
:104E500012441494FEF738FE002818BFFBF7EAFD51
:104E60004FF4FA700F9040F25060C2F200000EA9A9
:104E70000422FEF729FE002818BFFBF7DBFD40F2F5
:104E80005060C2F200000EA90822FEF71DFE0028A5
:104E900018BFFBF7CFFD00204FF40051CDE90610FD
:104EA0004FF000710590CDE90300CDE90100CDE997
:104EB0000800CDE90A10CDE90C0040F25060C2F2C2
:104EC000000001A9FEF72AF8002818BFFBF7B2FD81
:104ED00040F25064C2F2000420460021FFF72AF895
:104EE00020460421FFF726F820460821FFF722F884
:104EF00020460021FEF722F920460421FEF71EF984
:104F000020460821FEF71AF92046FEF76BFD1CB07B
:104F100010BD000010B592B040F29C600024C2F2B7
:104F200000004FF08041C0E900140321CDE90914CD
:104F300001214FF48052CDE90B14CDE90F1409A9DA
:104F40000894CDE90644CDE90444CDE90244CDE915
:104F50000044C0E9024204618461CDE90D4411942A
:104F6000FEF7E8FA002818BFFBF764FD40F29C60EA
:104F7000C2F2000006A906940894FEF76FF8002814
:104F800018BFFBF757FD0020CDE90400CDE9000074
:104F900002908DF80C0040F29C60C2F2000069465D
:104FA000FEF726F8002818BFFBF744FD12B010BD2D
:104FB00010B592B040F2E86040F200410024C2F225
:104FC0000000C4F20001C0E900140321CDE9091476
:104FD00001214FF48052CDE90B14CDE90F1409A93A
:104FE0000894CDE90644CDE90444CDE90244CDE975
:104FF0000044C0E9024204618461CDE90D4411948A
:10500000FEF798FA002818BFFBF714FD40F2E8609D
:10501000C2F2000006A906940894FEF71FF80028C3
:1050200018BFFBF707FD0020CDE90400CDE9000023
:1050300002908DF80C0040F2E860C2F20000694670
:10504000FDF7D6FF002818BFFBF7F4FC12B010BD27
:1050500010B59CB0002401A834211B94CDE919445B
:10506000CDE91644CDE91444CDE91244CDE910440C
:10507000CDE90E44FBF704F940F2347043F20041ED
:10508000C2F20000C4F2010141F27B52C0E90014F7
:10509000C0E90242C0E904448461FEF7DBF800285D
:1050A00018BFFBF7C7FC4FF48050189040F23470E3
:1050B000C2F2000018A9FEF72DF9002818BFFBF76F
:1050C000B9FC40F23470C2F20000FEF7FDFE002889
:1050D00018BFFBF7AFFC40F234700024C2F20000AE
:1050E00015A9CDE915441794FDF7B8FF002818BF9E
:1050F000FBF7A0FC60200E904FF4FA70CDE90F048E
:1051000040F23470C2F200000EA90022CDE9114431
:10511000CDE91344FEF7D8FC002818BFFBF78AFC42
:1051200040F23470C2F200000EA90422FEF7CCFC5B
:10513000002818BFFBF77EFC40F23470C2F200007A
:105140000EA90822FEF7C0FC002818BFFBF772FC6E
:1051500000204FF40051CDE906104FF0007105908A
:10516000CDE90300CDE90100CDE90800CDE90A1041
:10517000CDE90C0040F23470C2F2000001A9FDF745
:10518000CDFE002818BFFBF755FC40F23470C2F288
:105190000000FEF727FC1CB010BD000080B540F2F7
:1051A000807043F60001C2F20000C4F20101002346
:1051B0004FF00C0C4FF4E12280E80E00C0E90333FD
:1051C000C0E905C3C0E90733C0E90933FFF72EF88A
:1051D000002818BFFBF72EFC40F28070C2F20000DE
:1051E0000021FEF7DDFF002818BFFBF723FC40F28B
:1051F0008070C2F200000021FEF78CFF002818BF6B
:10520000FBF718FC40F28070C2F20000FEF766FF68
:10521000002808BF80BDBDE88040FBF70BBC000044
:1052200080B540F6140044F60001C2F20000C4F25A
:10523000000100234FF00C0C4FF4E13280E80E0027
:10524000C0E90333C0E905C3C0E90733C0E9093346
:10525000FEF7ECFF002818BFFBF7ECFB40F614004C
:10526000C2F200000021FEF79BFF002818BFFBF7E9
:10527000E1FB40F61400C2F200000021FEF74AFFF5
:10528000002818BFFBF7D6FB40F61400C2F200005E
:10529000FEF724FF002808BF80BDBDE88040FBF773
:1052A000C9BB0000FEE7000040F23C00C2F2000073
:1052B00090ED001AB1EE080AB4EE401AF1EE10FAC1
:1052C00002DD80ED000A08E0B9EE080AB4EE401AEB
:1052D000F1EE10FAB8BF80ED000A90ED011AB1EEC0
:1052E000080AB4EE401AF1EE10FA03DD80ED010A6F
:1052F00009E000BFB9EE080AB4EE401AF1EE10FA68
:10530000B8BF80ED010A90ED021AB1EE080AB4EEC2
:10531000401AF1EE10FA03DD80ED020A704700BF7B
:10532000B9EE080AB4EE401AF1EE10FAB8BF80EDFB
:10533000020A7047FEE7000040F248004DF20A7290
:10534000C2F20000C3F6234241F26F23026141F230
:105350006F22C3F603234FF07A5CC3F60332436136
:10536000C0F818C04CF2AC5C4263836345F2EC12A7
:105370004DF20A730021C3F2277CC3F63852C3F6FC
:10538000A333C0E90011C0E90211C161C0E90811ED
:10539000C0E90A110163C0F83CC0C0E91011C0E9BE
:1053A0001211C0E91411C0E91623C0E91811816671
:1053B00070470000704700007047000000000000C8
:1053C00010B52DED048BB0EE408AFBF791FA40F258
:1053D0001010C2F2000080ED000A38EE400A00F022
:1053E00051F840F24004C2F2000484ED000AFFF7D5
:1053F0005BFF40F2080040F20401C2F20000C2F27A
:1054000000010068096894ED008A484300EE100A24
:10541000B8EEC09AFBF758FA40F6B000C2F20000AE
:1054200090ED001A29EE000A30EE410A10EE100A43
:10543000FBF7B9F841EC100B9FED0F1B01F0C4F81E
:1054400051EC100BFBF7C2F89FED0D0A01EE100AAC
:1054500071EE000AB5EE401AF1EE10FAA8BFF0EEB8
:10546000410AB0EE480ABDEC048BBDE8104000F0E4
:1054700097BE00BF00BF00BF00000060FB211940C5
:10548000DB0FC94040F26C00C2F20000B0EE401ADF
:1054900090ED080A90ED032A90ED043A90ED054A4C
:1054A00030EE010A90ED065A20EE044A23EE013A4E
:1054B00031EE422A33EE043A25EE022A32EE032A76
:1054C0009FED0E3A9FED0E4AB4EE430A80ED021AAC
:1054D000BDEEC22AF1EE10FAB8BFB0EE430AB4EE48
:1054E000440AF1EE10FAB8BFB0EE404AB8EEC20A74
:1054F00080ED084A80ED031A704700BF00803BC56D
:1055000000803B45FCF7F0BD4EF68850CEF200001F
:10551000016841F4700101607047000040F29C6036
:10552000C2F20000FEF778B910B540F29C64C2F2F6
:10553000000420463C21FEF70FF92046BDE810404C
:10554000FDF780BD40F2E860C2F20000FEF764B9EA
:1055500010B540F2E864C2F2000420463C21FEF798
:10556000FBF82046BDE81040FDF76CBD80B540F665
:10557000FF330268C4F2000343F2FF3C9842C4F2D6
:10558000010C0BDD60452FDC40F60043C4F2000344
:10559000984235D042F600432EE000BFB0F1804F74
:1055A0002ED040F20043C4F20003984228D040F6C7
:1055B0000003C4F20003984222D0604526DC40F28A
:1055C000FF73C4F20003984236DD40F60003C4F2D4
:1055D0000003984244D040F60043C4F200039842CE
:1055E0003ED042F6004337E045F20003C4F2010327
:1055F000984205D043F20043C4F201039842DCD143
:105600004B6822F070021A436045D8DD44F2FF3344
:10561000C4F20103984217DD44F20043C4F20103CF
:1056200098421DD045F20003C4F20103984217D0FE
:1056300044F6000310E000BFB0F1804F10D040F2FC
:105640000043C4F2000309E043F20043C4F2010343
:10565000984205D044F20003C4F20103984203D1FA
:10566000CB6822F440721A434B6922F0800E8A689C
:1056700043EA0E03D1F800C00360C262A0F1804289
:10568000A2F596324FEAB222092AC0F828C008D8FB
:10569000012303FA02F240F2E5231A421CBF096912
:1056A0000163012141610169C90708BF80BD01692A
:1056B00021F00101016180BDD0F808C011432CF434
:1056C0007F4C41EA032141EA0C01816070470000F0
:1056D00080B5816A0A070DD4CA0716D18A071FD47C
:1056E0004A0728D4CA0631D48A063AD44A0658D57D
:1056F00042E000BF0268D0F838C0536823F400438A
:1057000043EA0C035360CA07E8D00268D0F82CC003
:10571000536823F4003343EA0C0353608A07DFD550
:105720000268D0F830C0536823F4803343EA0C0396
:1057300053604A07D6D50268D0F834C0536823F4C2
:10574000802343EA0C035360CA06CDD50268D0F823
:105750003CC0936823F4805343EA0C0393608A06A9
:10576000C4D50268D0F840C0936823F4005343EADC
:105770000C0393604A0614D50268D0F844C05368FD
:10578000BCF5801F23F4801343EA0C03536008D157
:10579000D2F804C0D0F848E02CF4C00343EA0E036A
:1057A0005360090658BF80BD0168C06C4A6822F486
:1057B00000221043486080BDB0B582B0044600208E
:1057C000C4F89000FCF750FA216805460A681207F1
:1057D00037D56FF07E4C20464FF4001100222B4647
:1057E000CDF800C000F000FA50B300BF206850E8C8
:1057F000000F216820F0800041E80002DAB1206843
:1058000050E8000F216820F0800041E8000292B1CA
:10581000206850E8000F216820F0800041E8000275
:105820004AB1206850E8000F216820F0800041E86C
:105830000002002ADAD12020C4F8880060E000BF0E
:1058400021680868400761D56FF07E4C20464FF410
:10585000800100222B46CDF800C000F0C5F90028D9
:1058600054D000BF206850E8000F216820F49070E9
:1058700041E80002E2B1206850E8000F216820F4FE
:10588000907041E800029AB1206850E8000F21684A
:1058900020F4907041E8000252B1206850E8000FF7
:1058A000216820F4907041E80002002ADAD100BF9C
:1058B000206850E8020F216820F0010041E8020250
:1058C000DAB1206850E8020F216820F0010041E8B9
:1058D000020292B1206850E8020F216820F0010016
:1058E00041E802024AB1206850E8020F216820F026
:1058F000010041E80202002ADAD12020C4F88C001D
:105900000320002184F8841002B0B0BD2020C4F828
:105910008800C4F88C000020E0662067002184F82D
:10592000841002B0B0BD000070B504462269D4E90D
:10593000021300680A436169E6691143026846F68A
:10594000F315CCF6FF7531432A40114301604168DD
:1059500048F2000C21F4405119434160A269C4F29D
:10596000000C60451CBF216A0A4381684FF2FF4367
:10597000C1F2FF13194011438160C16AD4F824E0D9
:1059800021F00F0141EA0E01C16244F6FF71C4F239
:10599000000188424FF0100318DC44F20041C4F2C9
:1059A0000001884228D044F60001C4F20001884278
:1059B0002AD044F60041C4F20001884242D141F2AB
:1059C0008801C4F2020109688B0933E045F2000145
:1059D000C4F2000188421FD0604525D043F6000183
:1059E000C4F2010188422DD141F28801C4F20201C2
:1059F0000B6879A222E000BF41F28801C4F20201E3
:105A000009688B0816E000BF41F28801C4F2020168
:105A100009680B090EE000BF41F28801C4F20201DF
:105A200009680B0A06E000BF41F28801C4F20201D6
:105A300009688B0A47F26012C0F6000203F0030106
:105A400052F82130604542F20040C0F2F40015D017
:105A5000B6F5004F24D1082B4FF0010100F2B380BE
:105A6000DFE803F0065E6CB164B1B1B16A0000BF5B
:105A7000FCF778FF002856D15CE000BF082B4FF000
:105A8000010100F2A080DFE803F0059E259E1D9E27
:105A90009E9E2300FCF766FFC0B1D4F824E019E015
:105AA000082B4FF0010100F28E80DFE803F005655E
:105AB000738C6B8C8C8C7100FCF754FF00285ED1CA
:105AC00064E000BFFCF77AFF0028E6D100217AE00D
:105AD0004FF4004047F24811C0F6000131F81E10A3
:105AE0006268B0FBF1F002EB420188424FF0010125
:105AF00069D31303984266D8010E000210EB5200DE
:105B000041F100010023FAF783FB4FF60052A0F5A4
:105B10004071C0F20F0291424FD3012153E000BF08
:105B2000FCF736FF30B1D4F824E007E0FCF746FF7D
:105B30000028F8D1002146E04FF4004047F2481118
:105B4000C0F6000131F81E106268B0FBF1F0510898
:105B500001EB4000B0FBF2F04FF6EF72A0F1100144
:105B6000914207D84FF6F0710140C0F3420008445B
:105B700023E000BF012126E0FCF70AFF30B1D4F892
:105B800024E007E0FCF71AFF0028F8D100211AE012
:105B90004FF4004047F24811C0F6000131F81E10E2
:105BA0004FF6EF72B0FBF1F0616800EB5100B0FB13
:105BB000F1F0A0F11001914204D82168C8600021E1
:105BC00001E000BF01214FF00110A066002208464D
:105BD0006267A26770BD00BF010000000400000002
:105BE00002000000080000002DE9F0418046006836
:105BF0001546C2690E461140891BB1FA81F1490967
:105C0000A94223D1069C2CB3611C29D1C169314022
:105C1000891BB1FA81F14909A94217D1C169314003
:105C2000891BB1FA81F14909A9420FD1C1693140FB
:105C3000891BB1FA81F14909A94207D1C1693140F3
:105C4000891BB1FA81F14909A942DFD00020BDE8E2
:105C5000F08100BFFCF708F80320BDE8F08100BF29
:105C60001F4607E0C0693040801BB0FA80F0400951
:105C7000A842EBD1FBF7F8FFC01BA04242D8D8F8EE
:105C8000000001684907EDD5402EEBD0802EE9D009
:105C9000C16909073AD4C1690905E3D54FF4006128
:105CA000016250E8000FD8F8001020F4907041E82D
:105CB0000002002A60D0D8F8000050E8000FD8F8A1
:105CC000001020F4907041E80002002A54D0D8F867
:105CD000000050E8000FD8F8001020F4907041E860
:105CE0000002002A48D0D8F8000050E8000FD8F889
:105CF000001020F4907041E80002EAB3D8F80000E8
:105D0000CFE700BF0320BDE8F08100BF082101629A
:105D100050E8000FD8F8001020F4907041E800021D
:105D2000002A00F09780D8F8000050E8000FD8F85B
:105D3000001020F4907041E80002002A00F08A80F0
:105D4000D8F8000050E8000FD8F8001020F4907048
:105D500041E80002002A7DD0D8F8000050E8000F8A
:105D6000D8F8001020F4907041E80002002A71D0A9
:105D7000D8F80000CCE700BF4FF6FE70CEF6FF70FB
:105D8000D8F8001051E8021FD8F80020014042E87E
:105D90000213F3B1D8F8001051E8021FD8F8002020
:105DA000014042E80213A3B1D8F8001051E8021FE5
:105DB000D8F80020014042E8021353B1D8F800108F
:105DC00051E8021FD8F80020014042E80213002BDE
:105DD000D6D1D8F86C0001282CD1D8F8000050E8B2
:105DE000000FD8F8001020F0100041E800020AB3BC
:105DF000D8F8000050E8000FD8F8001020F010008C
:105E000041E80002B2B1D8F8000050E8000FD8F81D
:105E1000001020F0100041E800025AB1D8F800004C
:105E200050E8000FD8F8001020F0100041E8000200
:105E3000002AD2D120200021C8F88C00C8F86C10AC
:105E4000C8F87410C8F89000032088F88410BDE8E2
:105E5000F08100BF4FF6FE70CEF6FF70D8F800104C
:105E600051E8021FD8F80020014042E80213F3B1C4
:105E7000D8F8001051E8021FD8F80020014042E88D
:105E80000213A3B1D8F8001051E8021FD8F800207F
:105E9000014042E8021353B1D8F8001051E8021F44
:105EA000D8F80020014042E80213002BD6D1D8F8E0
:105EB0006C0001282CD1D8F8000050E8000FD8F869
:105EC000001020F0100041E800020AB3D8F80000EA
:105ED00050E8000FD8F8001020F0100041E8000250
:105EE000B2B1D8F8000050E8000FD8F8001020F048
:105EF000100041E800025AB1D8F8000050E8000F45
:105F0000D8F8001020F0100041E80002002AD2D199
:105F10002020C8F88C0000200821C8F86C00C8F8C0
:105F20007400C8F8901088F884000120BDE8F08162
:105F3000B0B540F2E864C2F2000420463C21FDF70F
:105F40000BFC2046FDF77EF8206840F2B404C2F254
:105F50000004406A216A6062411A0BB20D46A26ACF
:105F600041F2010E13F5006FB8BF75444EF6FF7C89
:105F7000B3F5006FC8BF01EB0C0529B26163811A4C
:105F800021EAE1711144091A43F6FF731944994358
:105F900020620844801A410000EE101A9FED0E1A8C
:105FA000B8EEC00A20EE010A9FED0C1A206020EE28
:105FB000010AB5EE001A20EE010ABDEEC00A84ED1A
:105FC0000B0AB8EEC00A00F00FF8606ABDEEC00A16
:105FD00084ED0C0AB0BD00BFDB0F494000008039E2
:105FE000FEE700000000000080B510EE100AFAF78E
:105FF000DAFA41EC100B9FED0C1B00F0E5FA51ECC6
:10600000100BFAF7E3FA9FED0A0A01EE100A31EEDF
:10601000000AB5EE401AF1EE10FAA8BFB0EE410A40
:1060200080BD00BF00BF00BF00000060FB21194021
:10603000DB0FC94094B0FCF765F800240020CDE9DF
:106040000B44CDE90944CDE90744FCF7F7F84FF4D8
:106050008071099140210A91042102200F9155215C
:106060000690CDE90D00CDE91010CDE9120006A88B
:10607000FCF7E2FC20B1EFF3108072B6FEE700BF40
:106080000F2001900320CDE9020401A80421CDE9ED
:106090000444FCF7DDFA28B1EFF3108072B600BFBC
:1060A000FEE700BFFEF752FDFEF7C4FCFEF730FE30
:1060B000FFF774F8FEF76EFEFEF7CAFFFEF77AFBF5
:1060C000FEF7F4FBFEF7B8FDFEF7ECFDFFF7A8F8CE
:1060D000FEF7ECFCFEF756FCFEF710FDFEF71AFF8C
:1060E000FEF766FF1D2000210022FCF76BF81D2043
:1060F000FCF758F81C2000210022FCF763F81C2054
:10610000FCF750F840F22810C2F20000FAF7D2FB78
:1061100040F24410C2F20000FAF7CCFB40F26010EB
:10612000C2F20000FAF7C6FB40F20404C2F2000417
:1061300094ED020AFAF7E4FCD4E90001FAF780FCD6
:10614000FFF7F2F9FFF704FA4FF090404FF4806147
:1061500001220126FBF782FD40F60000C4F6000094
:106160004FF400710122FBF779FD40F2145440F224
:106170002005C2F20004C2F2000501E0FFF7D8FEDC
:10618000204629460696FAF715FC0028F6D19DED23
:10619000060AB8EEC00AFFF713F9EFE700000000A7
:1061A0002DE9F04F81B02DED088B82B040F20C0745
:1061B000C2F2000797ED001ABEEE002A21EE028A15
:1061C000B4EE408AF1EE10FA0CDCB6EE002A21EEB5
:1061D000021AB4EE401AF1EE10FAB8BFB0EE410A5E
:1061E000B0EE408A10EE900AFAF7DDF941EC100BA0
:1061F0009FEDAB1B00F0E8F951EC100BFAF7E6F954
:106200009FEDAF0A01EE100A18EE104A31EE009A27
:10621000B5EE401A84F00040F1EE10FAA8BFB0EEDF
:10622000419AFAF7C0F9054619EE100A0E46FAF738
:10623000BAF941EC180BB0EE480AF0EE680A00F02B
:1062400047FA51EC100B2A463346FAF7CBF8FAF727
:10625000BDF940F21816C2F2000630602046FAF787
:10626000A2F9B0EE480AF0EE680A04460D4600F0C6
:1062700047F951EC100B22462B46FAF7B3F8FAF720
:10628000A5F940F2201197ED008AC2F2000196EDC7
:1062900000AAB6EE000A086028EE00BA40F2141117
:1062A0003AEE0B9AC2F2000181ED009AFAF77BF9FF
:1062B00082461AEE100A8B46FAF775F99FED7A0BB3
:1062C000044601900D46009153EC102B5046594660
:1062D000FAF788F822462B46FAF77EF89FED740B02
:1062E00054EC105B2A462346FAF77CF880461BEEF6
:1062F000100A8946FAF757F942464B4606460F46BA
:10630000F9F7C9FFFAF762F940F21C119FED6A0B29
:10631000C2F200010AEE100A086053EC102B50463E
:106320005946FAF75FF8DDE90032FAF755F82A46E0
:106330002346FAF757F802460B4630463946F9F736
:10634000AAFFFAF743F940F22411C2F200019FEDCF
:106350005D0A0860B5EE409A40F21C01F1EE10FAB9
:10636000C2F20001B0EE401A0ADB91ED001AB4EE61
:10637000491AF1EE10FAB8BFB0EE419AB0EE491AE0
:10638000B5EE40AA04EE100AF1EE10FAB0EE402A83
:106390000ADB91ED002AB4EE4A2AF1EE10FAB8BFFA
:1063A000B0EE42AAB0EE4A2AB5EE404AF1EE10FA3B
:1063B000B0EE403A0ADB91ED003AB4EE443AF1EE29
:1063C00010FAB8BFB0EE434AB0EE443A81EE081A74
:1063D00082EE082A83EE083AB7EE004A40F27C10BB
:1063E000B0EE405AC2F20000B4EE441AF1EE10FAD8
:1063F000C8BFB0EE441AB5EE401AF1EE10FAC8BFAD
:10640000B0EE415A80ED005AB4EE442A40F28010BA
:10641000F1EE10FAC8BFB0EE442AB5EE402AB0EE55
:10642000401AC2F20000F1EE10FAC8BFB0EE421AF4
:1064300080ED001AB4EE443A40F28410F1EE10FA06
:10644000C8BFB0EE443AB5EE403AC2F20000F1EEF9
:1064500010FAC8BFB0EE430A9FED1B2A80ED000A78
:1064600040F25060C2F2000025EE023A006821EED0
:10647000021A20EE020ABCEEC33ABCEEC11ABCEE10
:10648000C00A80ED0D3A80ED0E1A80ED0F0A02B0C1
:10649000BDEC088B01B0BDE8F08F00BF00BF00BFAE
:1064A00000000060FB211940AA4C58E87AB6FB3F77
:1064B000000000000000E03FAA4C58E87AB6FBBF9D
:1064C000DB0FC9400000000000E0AB4503B40198B9
:1064D0004100009850EAC12018BF04204A0D18BF9F
:1064E00040F0010040F2FF72B2EB515F08BF40F094
:1064F0000200012808BF052002B07047000000001C
:1065000010B52F499FED2C1B2DED020B84B0059883
:1065100020F000408842D8BF9DED040B2DDD2949B5
:10652000884209D1049840B94FF0010000F058FDAD
:1065300000F026FD06B010BD05DB9DED040B00F05C
:1065400013FD06B010BD68469DED040B00F024F964
:1065500010F0030004BF9DED021B9DED000B0CD05D
:1065600001280ED09DED021B9DED000B022817D0D7
:10657000012000F061FC06B010BD00F029FB06B060
:1065800010BD9DED021B9DED000B012000F054FCA1
:1065900051EC100B81F0004106B041EC100B10BD26
:1065A00000F016FB51EC100B81F0004106B041ECFD
:1065B000100B10BD000000000000000000000000F3
:1065C000FB21E93F0000F07F10B52DED040B86B0F4
:1065D0009DED060B10EE100A10EE901A8DED000BDB
:1065E000002818BF0120084320F00040C0F17F6060
:1065F00000F1E040C00F21D19DED080B10EE101A04
:1066000010EE900A8DED000B002918BF0121084300
:1066100020F00040C0F17F6000F1E040C00F0DD1DC
:1066200029490798B1EB400F04BF0698002842D0D3
:106630000998400004BF089800283CD09DED080B45
:1066400053EC102B9DED060B51EC100BFAF79FF855
:10665000CDE902019DED020B40F2FF7110EE900AB0
:106660008DED000B31EA105021D00798039900F00E
:10667000004001F00041884219D09DED080B8DEDDE
:10668000040B9DED020B8DED000B10EE900A0599A9
:1066900061F31E0005909DED041B9DED020B51EC76
:1066A000110B53EC102BF9F79AFECDE902019DED89
:1066B000020B0AB010BD012000F092FC0AB0BDE848
:1066C000104000F05DBC00000000E0FF0000000092
:1066D00010B52F499FED2C1B2DED020B84B00598B2
:1066E00020F000408842DCBF00209DED040B32DD2D
:1066F0002849884209D1049840B94FF0010000F0C0
:106700006FFC00F03DFC06B010BD05DB9DED040BF9
:1067100000F02AFC06B010BD68469DED040B00F0A9
:106720003BF810F0030011D0012818D09DED021B9A
:106730009DED000B02281AD000F04AFA51EC100B24
:1067400081F0004106B041EC100B10BD9DED021B25
:106750009DED000B012000F06FFB06B010BD9DED1C
:10676000021B9DED000B00F033FA06B010BD0120B6
:1067700000F062FB51EC100B81F0004106B041ECDF
:10678000100B10BD00000000000000000000000021
:10679000FB21E93F0000F07F2DE9F14F04462DED8C
:1067A000020B2DED088B8AB09FEDE70B80ED020BFD
:1067B000139EE74826F0004585420ADC9DED120B4A
:1067C000002084ED000B0AB0BDEC088B03B0BDE8DF
:1067D000F08FE0489FEDE0AB9FEDE1BBA84247DDC5
:1067E000E14F9FEDE39B9FEDE48B9DED120B53EC8E
:1067F0001A2B51EC100B002E1CDDF9F7EDFD41ECCE
:10680000100BBD4208D053EC1B2B51EC100BF9F7C9
:10681000E3FDC4E900010BE053EC192B51EC100B24
:10682000F9F7DAFD53EC182BF9F7D6FDC4E90001AE
:106830000120C8E7F9F72FFD41EC100BBD4208D04D
:1068400053EC1B2B51EC100BF9F725FDC4E90001AB
:106850000BE053EC192B51EC100BF9F71CFD53EC2A
:10686000182BF9F718FDC4E900014FF0FF30AAE733
:10687000C348A84279DB9DED120B51EC100B00F0E0
:10688000B5FB41EC180B9FEDC00B53EC102BF9F747
:10689000A9FD9FEDBF1B53EC112BF9F7FCFCF9F799
:1068A000E9FF0746F9F7C8FF41EC190B53EC1A2B27
:1068B000F9F798FD53EC182BF9F791FD41EC180B03
:1068C00053EC1B2B51EC190BF9F78CFDDFF8C8A228
:1068D00041EC100B4FEA15580125FA4453EC102BEC
:1068E00051EC180BF9F778FD032DC4E900013DD0F8
:1068F000C1F30A5005EB4511A8EB000011398142A4
:1069000034DA0AEB051BB0EE48AA9BED000BF0EE63
:1069100068AA53EC102B51EC190BF9F763FD41EC0D
:106920001B0B51EC1A0B53EC1B2BF9F755FD41ECEB
:10693000180B51EC1A0B53EC182BF9F74DFD53ECD7
:106940001B2BF9F749FD9BED020B41EC1A0B53ECA5
:10695000102B51EC190BF9F745FD53EC1A2BF9F7F5
:106960003BFD41EC100B6D1CB8E70EE0002EA8BFFC
:106970003846BFF628AF94ED000B51EC100B81F0B8
:106980000041C4E9000178421DE7C6F3130040F45A
:10699000801EC6F30A50A0F2F530471100F01F0523
:1069A000C5F12000DDF848B008900020069007905F
:1069B0000520EC467949002D07EB0002794408BF19
:1069C00051F8221009D051F8223001EB8201AB407E
:1069D0004A68089922FA01F11943A1FB0E26A1FB8E
:1069E0000B131A449A4234BF0123002303EB060819
:1069F0000CEB8003D3E901A60E448E4234BF012183
:106A0000002192448A4411B1924502D903E0924593
:106A100001D2012100E00021C3E901A641444CF864
:106A20002010011EA0F10100C4DC029800F100500A
:106A3000850F0298DDE903678000DDF81480F9F71F
:106A4000FBFE41EC1A0B3046F9F707FF9FED541B94
:106A500053EC112BF9F7C6FC41EC1B0B3846F9F748
:106A6000FCFE9FED511B53EC112BF9F7BBFC41ECE5
:106A7000180B4046F9F7F1FE9FED4D1B53EC112B1F
:106A8000F9F7B0FC41EC190B51EC180B53EC192B36
:106A9000F9F701FC53EC1B2BF9F7FDFB53EC1A2B18
:106AA000F9F7F9FBCDE90801002008909DED080BEE
:106AB00053EC1A2B51EC100BF9F78EFC53EC1B2BFB
:106AC000F9F78AFC53EC182BF9F786FC53EC192BD9
:106AD000F9F785FC9FED381B53EC112BF9F782FC7D
:106AE0009FED370B41EC180B53EC102B9DED080B71
:106AF00051EC100BF9F776FC53EC182BF9F7CBFBA4
:106B00009FED310B41EC180B53EC102B9DED080B56
:106B100051EC100BF9F766FC53EC182BF9F7BBFBA3
:106B200041EC100B139810F0004F06D06D4251EC61
:106B3000100B81F0004141EC100B284684ED000B56
:106B400041E600000000000000000000000000001E
:106B5000FB21E93F7CD9024000004054FB21F93F72
:106B60003163621A61B4D03DFB21F93F000000009F
:106B70000000601A61B4D03D7370032E8A19A33BE4
:106B8000FB2139410000000083C8C96D305FE43F3C
:106B9000000000000000E03F5A070000A8060000C7
:106BA000000000000000103E000000000000103C4B
:106BB000000000000000103A182D4454FB21F93D5C
:106BC0003326A611460B113C00000054FB21F93D71
:106BD00010B52DED040B2DED088B82B0B0EE419A6F
:106BE000F0EE619A0B9820F000449FED4BABB4F1AE
:106BF000795F11DA9DED0A0B51EC100BF9F73AFEB3
:106C0000002801BFB0EE4A0AF0EE6A0A02B0BDECFD
:106C1000088B04BF04B010BD9DED0A0B53EC102B84
:106C200051EC100BF9F7DEFB41EC180B3C48062148
:106C3000B0EE480AF0EE680A784400F081F853ECB0
:106C4000182B51EC100BF9F7CDFB9DED0A0B41EC25
:106C50001B0B53EC192B51EC100BF9F7C3FB41EC58
:106C6000190B53EC1B2B51EC180BF9F7BBFB53EC36
:106C7000192BF9F7B1FB9FED2C0B41EC190B53ECE1
:106C8000102B51EC180BF9F7ADFB41EC100B284819
:106C9000844210DA53EC192B51EC100BF9F79CFBE2
:106CA00053EC1A2BF9F79BFB41EC100B02B0BDEC37
:106CB000088B04B010BD1F48A042BCBF9FED1E1B37
:106CC0008DED001B06DBA4F5001001900020009064
:106CD0009DED001B51EC100B53EC112BF9F77CFBD5
:106CE0009DED000B41EC180B53EC102B51EC1A0BE3
:106CF000F9F772FB41EC1A0B53EC192B51EC180B02
:106D0000F9F76AFB53EC1A2BF9F769FB41EC100B0E
:106D1000CCE7000000000000000000000000F03F91
:106D2000CC03000000000000000000000000E03F75
:106D30003333D33F0000E93F000000000000D23FA2
:106D400070B504462DED028B4D1E00EBC500B0EE74
:106D5000408AF0EE608A90ED000B35F0060017D007
:106D600053EC182B51EC100BF9F73CFB41EC100BDA
:106D70006D1E04EBC50090ED001B51EC100B53ECA5
:106D8000112BF9F788FA41EC100B35F00600E7D12A
:106D9000022D36D0042D1CD0062D1CBFBDEC028B5D
:106DA00070BD53EC182B51EC100BF9F71BFB94ED55
:106DB0000A1B53EC112BF9F76EFA53EC182BF9F769
:106DC00011FB94ED081B53EC112BF9F764FA41EC1D
:106DD000100B53EC182B51EC100BF9F703FB94ED4F
:106DE000061B53EC112BF9F756FA53EC182BF9F755
:106DF000F9FA94ED040B53EC102BF9F74CFA41EC33
:106E0000100B53EC182B51EC100BF9F7EBFA94ED37
:106E1000021B53EC112BF9F73EFA53EC182BF9F740
:106E2000E1FA94ED001B53EC112BF9F734FABDECA9
:106E3000028B41EC100B70BD31B504462DED040BF7
:106E40002DED0A8BB0EE41BAF0EE61BA0B989DEDD4
:106E50000A0B20F00040B0F1795F0DDA51EC100B15
:106E6000FFF734FB042808BF00F09AF89DED0A0BE9
:106E7000BDEC0A8B05B030BD53EC102B51EC100B60
:106E8000F9F7B0FA41EC180B9DED0A0B53EC182BF7
:106E900051EC100BF9F7A6FA41EC190B2C48B0EEA7
:106EA000480AF0EE680A05217844FFF749FF9FED94
:106EB0002ACBB0EE40AAF0EE60AA9CB353EC1C2B98
:106EC00051EC190BF9F78EFA41EC1C0B53EC1A2B11
:106ED00051EC190BF9F786FA9FED210B41EC190BD8
:106EE00053EC102B51EC1B0BF9F77CFA53EC192BDC
:106EF000F9F772FA53EC182BF9F774FA53EC1B2BD1
:106F0000F9F76AFA53EC1C2BF9F766FA9DED0A1BA8
:106F100053EC112BF9F763FABDEC0A8B05B041EC89
:106F2000100B30BDFFE753EC1A2B51EC180BF9F79F
:106F300059FA53EC1C2BF9F7AEF953EC192BF9F76E
:106F400051FA9DED0A1B53EC112BF9F7A4F9E3E775
:106F50005C02000000000000495555555555C5BF5D
:106F6000000000000000E03F10B553EC102B51EC86
:106F7000100BF9F790F941EC100B10BD0000000068
:106F80009FED050B10B553EC102B51EC100BF9F7DE
:106F90009BFA41EC100B10BD000000000000000047
:106FA0009FED050B10B553EC102B51EC100BF9F7BE
:106FB00019FA41EC100B10BD000000000000001099
:106FC00002E008C8121F08C1002AFAD170477047B2
:106FD000002001E001C1121F002AFBD17047000010
:106FE00001490860704700000000002082B0CDE930
:106FF000000121F0004001909DED000B02B051EC2A
:10700000100B7047000000004C5555555555A53FD5
:107010007751C1166CC156BF9015CB19A001FA3E2D
:10702000AD529C804F7E92BEC4B1B4BD9EEE213E57
:10703000D43888BEE9FAA8BD00004054FB21F93FCE
:107040003163621A61B4D03D0000601A61B4D03D72
:107050007370032E8A19A33B0000002E8A19A33BEC
:10706000C14920259A837B39000000000000000000
:107070006E83F9A22915444ED15727FCC0DD34F5A3
:10708000999562DB4190433CAB6351FE61C5BBDE29
:107090003A6E24B7E0D24D42EA2E49061C92D1093D
:1070A0001CEB1DFE3EA729B1F53582E88444BB2EBA
:1070B00026709CE9417E5FB439D69139F439538307
:1070C0008B5F849C3B28F9BDFF97F81F0F9805DE66
:1070D0008B112FEF1F6D0A5ACF7E366DB709CB2764
:1070E000663F464F2DEA5F9EC7BA27757BF1E5EBF9
:1070F000F739073DEA92528AB15FFB6B085D8D1F3D
:107100004630035600000000A6F810111111813F0F
:10711000D561C119A0012ABF7DFEB157E31DC73E4D
:10712000EB9C2B8AE6E55ABE7CD5CF5A3AD9E53D91
:107130000000000000000000010203040607080927
:107140000000000001020304010002000400060028
:1071500008000A000C001000200040008000000120
:107160000000000004000000020000000800000011
:1071700001010103070100000804020408010101E4
:10718000A07100080000002020000000C06F00086F
:10719000C071000820000020980C0000D06F00088B
:1071A000000000000100000001000000000040415C
:1071B00010000000010000000024F4000000404125
:04000005080001D915
:00000001FF
